:03000000020253A6
:03000300D2C12245
:05000600D2C0D2C122AE
:03000B0002521C82
:10000E00E5F06010C3EC13FCED13FDEE13FEEF13E1
:05001E00FFD5F0F02207
:030023000297271A
:10002600CD30E11520E00FC083C08288828C83CD5D
:0C003600F0D082D08322CDF222CDF62241
:10004200CB30E11520E00FC083C08289828A83CB46
:0C005200F0D082D08322CBF322CBF72227
:10005E00ED30E11320E00EC083C08288828C83E0F5
:10006E00D082D08322E2226405700EC083C08288C3
:0B007E00828C8393D082D08322E62284
:1000890088F0A8817404C0E0C0F018E6C0E008E672
:10009900C0E00886F018188001A3E0C608D5F0F979
:0200A900F8223B
:1000AB00EEC0E0EFC0E088F0E58124FDF8ECC6C0BF
:0900BB00E008EDC6C0E0A8F02247
:0C00C400E0A3FCE0A3FDE0A3FEE0FF22AF
:0C00D000ECF0A3EDF0A3EEF0A3EFF022A3
:0C00DC00E208FCE208FDE208FEE2FF2260
:0C00E800E309FCE309FDE309FEE3FF224D
:0C00F400ECF309EDF309EEF309EFF32241
:1001000075F004AA83AB82D083D082E493A3CAC5DE
:1001100083CACBC582CBF0A3CAC583CACBC582CB69
:08012000D5F0E8C082C0832283
:10012800120231C380021819E637F6DAF902022200
:10013800E0A3FEE0FFEF8DF0A4CFC5F0CCA42CFC2B
:09014800EE60038DF0A42CFE22F0
:10015100C2D1C2D5EE30E707D2D1D2D51201FEEC21
:1001610030E705B2D112020612017930D103120132
:10017100FE30D50312020622BC000EBE0032EF8D06
:10018100F08420D226FFADF0227B0075F008EF2F1E
:10019100FFEE33FEEB33FBEE9DEB9C4005FBEE9D4A
:1001A100FE0FD5F0E9E4CECDCBCC227EFF7FFF223E
:1001B100EDB410005022EE8DF084FEEF54F045F0C6
:1001C100C48DF084C4FCEF540FC445F0C48DF08499
:1001D100FFADF0E4CC4FFF22EE8DF08420D2CC7E37
:1001E10008CEC5F0CDCBEF2FFFED33FD10D7079B28
:1001F1005005D5F0F1229BFD0FD5F0EA22C3E49F13
:0D020100FFE49EFE22C3E49DFDE49CFC2270
:0C020E00EE30E707E4C39FFFE49EFE22F1
:10021A0074F9800674FA800274FCD083D082258136
:07022A00F581C082C08322B0
:0F023100E5D054182407F8E58124FCF97A04225B
:10024000EFB40A077F0D1202407F0A3099FDC29970
:030250008F992261
:0F025300758122E4787FF6D8FD75A0000257DD93
:0702620075850175C01B2228
:03026900C2C022EE
:05026C00C2C0D2C22255
:0A027100C20874017900F31207F5CA
:10027B00129672EF7901F3E314600B14601F146094
:06028B0040146053805492
:100291007900E3B40101D340077900E314F380440A
:0D02A10074067900F3803D7900E3B4060691
:0602AE001207F5E4FF2237
:1002B4007900E3FF121EA9EF7802F2E2B404037F8F
:1002C400042230081CE4FF227900E3B4060050073E
:1002D4007900E304F3800A74017900F380037F0456
:1002E400227900E3B4040302044E5013E3146020A3
:1002F4001470030203A6147003020409020692E3B5
:1003040024FB70030204AF14700302052902027B6C
:100314007B027A0079E17D057C15786912081D7FDE
:10032400017B027A0079E11295A99000DEE0700B5E
:100334007F027B057A15797A1295A99000DEE0FA9E
:10034400B4010B7F027B057A15798B1295A9900075
:10035400DEE0FAB4020B7F027B057A15799C1295D4
:10036400A99000DEE0FAB4030B7F027B057A1579CD
:10037400AD1295A99000DEE0FAB4040B7F027B0570
:100384007A1579BE1295A99000DEE0FAB4050280D0
:10039400030206927F027B057A1579CF1295A90292
:1003A400027B7B027A0079E17D057C1578E01208F6
:1003B4001D7F017B027A0079E11295A99000D5E0B6
:1003C400600790010CE0B401117B027A0079E17DB1
:1003D400057C1578F112081D801D9000D5E0FDE420
:1003E400C0E0C0057B027A0079E17D057C167802C5
:1003F40012081D158115817F027B027A0079E112B2
:1004040095A902027B7B027A0079E17D057C16784E
:100414001412081D7F017B027A0079E11295A990DC
:1004240000D3E0C0E0A3E0C0E07B027A0079E17D84
:10043400057C16782512081D158115817F027B0223
:100444007A0079E11295A902027B7B027A0079E1B4
:100454007D057C16783512081D7F017B027A0079B0
:10046400E11295A99000DAE0FAA3E0FBBA0004B423
:100474000001D34019C002C0037B027A0079E17DF8
:10048400057C16784612081D15811581800F7B02A4
:100494007A0079E17D057C16785612081D7F027B6F
:1004A400027A0079E11295A902027B9000DEE0FA5B
:1004B4006402600EEA64036009EA64046004EAB456
:0204C400051E13
:1004C6007901E3B401057900E314F37901E3B40398
:1004D6000280030206927900E304F302027B7B02A8
:1004E6007A0079E17D057C16786712081D7F017B0D
:1004F600027A0079E11295A99000DCE0C0E0A3E061
:10050600C0E07B027A0079E17D057C167846120808
:100516001D158115817F027B027A0079E11295A96A
:1005260002027B7B027A0079E17D057C16787812DF
:10053600081D7F017B027A0079E11295A99000DE01
:10054600E0B403030205EF500CE0601A1460431494
:10055600606C02066EE024FC700302061A14700337
:0605660002064502066ECC
:10056C009000D3E0C0E0A3E0C0E09000D5E0FDE453
:10057C00C0E0C0057B027A0079E17D057C167889A4
:10058C0012081D74FC2581F58102066E9000D3E0E3
:10059C00C0E0A3E0C0E09000D5E0FDE4C0E0C00501
:1005AC007B027A0079E17D057C16789A12081D741D
:1005BC00FC2581F58102066E9000D3E0C0E0A3E03B
:1005CC00C0E09000D5E0FDE4C0E0C0057B027A00FD
:1005DC0079E17D057C1678AB12081D74FC2581F53C
:1005EC0081807F9000D3E0C0E0A3E0C0E09000D514
:1005FC00E0FDE4C0E0C0057B027A0079E17D057C7A
:10060C001678BD12081D74FC2581F581805490006C
:10061C00D3E0C0E0A3E0C0E09000D5E0FDE4C0E092
:10062C00C0057B027A0079E17D057C1678CF120833
:10063C001D74FC2581F58180299000D3E0C0E0A3D6
:10064C00E0C0E09000D5E0FDE4C0E0C0057B027A9C
:10065C000079E17D057C1678E112081D74FC25817A
:0F066C00F5819000D5E0600790010CE0B4010C1F
:10067B0074209000E6F074419000E7F07F027B025B
:0A068B007A0079E11295A902027BC2
:080695007401791CF31207F552
:10069D00129672EF791DF3E3146012146027147033
:0D06AD000302073214700302074802074BD6
:1006BA00791CE3B40101D34008791CE314F302075F
:0E06CA004B7405791CF38079791CE3B40506A6
:0606D8001207F5E4FF2209
:0706DE00900115E0B40118C2
:1006E500791CE3FF122855EF781EF2E2B404037F6C
:0806F5000422300836E4FF2264
:1006FD001207F57F017B057A1A79321295A97F02CF
:10070D007B057A1A79431295A912965FE4FE7FFA5A
:10071D0012964712965F7E077FD01296471207F505
:10072D00E4FF228019791CE3B405005007791CE31E
:10073D0004F3800A7401791CF380037F0422791C71
:10074D00E314600E14601C14602A146038146046A3
:02075D008053C7
:10075F007B027A0079E17D057C1A785412081D809E
:10076F00427B027A0079E17D057C1A786512081DBB
:10077F0080317B027A0079E17D057C1A7876120848
:10078F001D80207B027A0079E17D057C1A78871223
:10079F00081D800F7B027A0079E17D057C1A78981D
:1007AF0012081D74069000E1F07F017B027A007938
:1007BF00E11295A97B027A0079E17D057C1A78A96F
:1007CF0012081D74059000E5F0049000E6F07F021A
:0C07DF007B027A0079E11295A902069DC8
:0A07EB0075D90275E90075F90022C6
:0607F5007F011294E022D6
:10080000A881058118EBC6C908CAC6CA08F67BFFCD
:10081000112ED0E0D0E0D0E0C082C08322D083D0BF
:1008200082EDC0E0ECC0E0E8C0E0C082C083E581BA
:10083000F8241EF58108E8C9CBF709EAF709EBF7B8
:1008400009770009E924F6FA75F000C2D5E924FC1D
:10085000F8E924F9F9ECC0E0E8C0E0D1E512005E67
:10086000FFE92409F9D0E0F8D0E0FCEF605020D592
:1008700074B4250AE4FB74FFFCF7D2D580D3D1FE13
:1008800080CFFF20F71CBCFF067014D2F380C2ECAF
:10089000C0F075F00AA42FD0F030F703F78001FC08
:1008A00080AFB7FF03EF80F4E780E57F00D1FE194A
:1008B0001709800DEF24D0B40A0040C68093B6FF1C
:1008C000EAE581C3941AF581E4FED0E0FFD082D03E
:1008D00083D0E004600ED083D0821581158115810C
:1008E000C082C08322900F78E49360256FA36006D6
:1008F000A350F5A380F293FF400442F080BEE4A32E
:10090000938F83F582E4C2D130F705B7FF027700F9
:100910007340A1D3A380D1EAC8FDE620F703FC8091
:1009200001F71A1AEDF88094D2D17F7880027F58AF
:10093000D17990100421CCBCFF05B7FF02805AC0CA
:10094000F08AF0EAC92419F583E8FEECC0E0D1E5AD
:1009500012005EFF601AC583C9C583F70B19E9C58C
:1009600083F908B800010CEE2404F9E7C39B70E09A
:10097000D0E0FCE5F024FDFAD0F08B82A98309EEEB
:10098000C394FBF583F805828004E7F60809D58255
:10099000F9A9831819C2F0414F8AF0EAC9F583E832
:1009A000FED1E512005EFF6013EEC8CE8D82D1FE4F
:1009B000AD82EEC8CE08B800EA0C80E7A983E5F066
:1009C00024FDFA01487F30D179900806C2F7D18919
:1009D000E8CAC9C88049D2F7EA147D0230F4047D20
:1009E0000424FEF8E68A83A88330E70DD2D1C3E45D
:1009F00096F618DDFAA8838000C2F7D179900A052F
:100A0000D189C9C8CAC9B1FF8015D179E618188043
:100A100004D1797425C2F7F70BCAC9C8CAC2F0E776
:100A2000FDE924002BF8B6300318DBFABB00080BF5
:100A300008BD00031B8013BDFF02800EEDC39BFEAB
:100A40004008600674305192EDFBEB70020148ECF7
:100A5000046023D39B401F601DFE7D2020F13830B1
:100A6000F3027D3030F023BD3018518E18EF30E6A0
:100A700001187111804030F03F71110B30F6390BC5
:100A80008036EF71111E30F6011E518E8028EE6007
:100A900005ED08F6DEFC2230F00771110B30F6018F
:100AA0000BE9FF2419F9E6F71918DBFAEDF719DE5F
:100AB000FCEFF92419F8CCCBEB700201481919E8C6
:100AC000C0E0E6FFD1E50909EFD16AD0E0F818DB14
:100AD000EE090901481A1AD181900F6CE6086002EC
:100AE0002406936023F7190B30E504E4A380F3EBAD
:100AF000C0E0743AF7E924FCF908901004D1891891
:100B0000D0E02405FBE92404C8CAC9E92419F88007
:100B1000AC08EFF68FF030F604743008F622619BD3
:100B2000C2F79159BFFF0261ADEF60F22481FF204F
:100B3000E73618040FD113EBC39F60124010FDFE7F
:100B40000BE89FF8742EC618C6DDFC18805DF4040F
:100B5000FD7E000DE824F9F880057430F6180BDDF1
:100B6000F9742EF60B188043F4FD7E070DBD0700C7
:100B70004016E9FD097430F709E9C39870F7EDF9FB
:100B800080087430F60E0B08DDF8742EF6080B0B97
:100B90007430F6D113E8C39BF88010E92419F87477
:100BA00030F618742EF6187B027E00B1AD414AC2B1
:100BB000F78002D2F79159BFFF0280F1BF000E7497
:100BC00030F618742EF6087E007B02800EEF24812A
:100BD000FF18742EC608C6EBFE1E0BD113E8C39B8C
:100BE000F8EFC0E0B1ADD113D0E0FFC0F0E8C39B97
:0E0BF000F8E730F704746580027445F618EFDC
:100BFE0020E704762B8004762DF4041875F00A8411
:100C0E002430F618E5F02430F6EB2404FBD0F0D1B6
:100C1E002918B1FF61ADC2F78002D2F7D2F2915915
:100C2E00BFFF0261ADE7B4FF037406F7BF7B004060
:100C3E0016EF248120E706C397600C500A74822FAA
:100C4E00C7C397F7020B2917020BBCD179ECC0E092
:100C5E00C0F018E63308E63392D5186033B4FF407F
:100C6E00E6C2E76009900FBCC2D17B078007900FE8
:100C7E00C3D2D17B06E493F709A3DBF97B0330D112
:100C8E000A742B30D502742DF70B09197C80A184C0
:100C9E00EAC0E074307A08F709DAFC097C81A17D9C
:100CAE00CAC0E0EA75F010A4CAABF075F04DA42BE3
:100CBE00FBE435F0FCEA2410FAEB34C5FBEC34D936
:100CCE00FCE6C2E7FF75F056A4F42411C5F0F43427
:100CDE00C58FF0A42AE5F03BE43CFBC0E0E9C0E0A0
:100CEE00E8C0E0EBC0E020E707800812112C801F5F
:100CFE00F404FB121411D0F0D0E0F8C0E0187583A4
:100D0E000418E6C0E008D583F930F7DF121288D058
:100D1E00E0F8D0E02408F9EED2E7CE33EF332482A8
:100D2E00FAECFBD0E0FCE4C3CB33CBCD33CDCE33EA
:100D3E00CE33DAF37A0875F00A8460062430F71998
:100D4E001A0CE5F02430F7198BF0740AA4FBAFF0FF
:100D5E008DF0740AA42FFDAFF050010F8EF0740ABF
:100D6E00A42FFE743035F0F719DADDE9240AF9D034
:100D7E00E0FAE9D39AFBECFF247FFFCAC9C824FD31
:100D8E00FAE9FD09EF046003120F2FEDF909EF04E4
:100D9E006003120F2FEDF9D0F0D0E0FC7B0722E7B5
:100DAE00B4FF027406700820F0010E8E838016C305
:100DBE009E400EF583603674300BF618D583FA809C
:100DCE002CF404F583C0E0E9C0E0E8C0E0F92B04A0
:100DDE00F8EEC0E0EFC0E009120F2DD583FAD0E097
:100DEE00FFD0E0FED0E0F8D0E0F9D0E0FD08D12948
:100DFE0018D2F07F2D20D10C7F2B20F5077F2020DD
:100E0E00F602C2F0228982E92419F98B83E6F719DA
:100E1E0018D583F9A982E92419F822E9F58224016B
:100E2E00F98B8330F22A20F027C2F2E608B42E02A4
:100E3E00D2F2D583F6E8C39BF88B8330F210E6B47A
:100E4E003005081BD583F7B42E07081B8006D2F297
:100E5E00E6F70908D583F9E9F8A98222BDFF051244
:100E6E000240800312002609071922E9CAC8E924A4
:100E7E0001F922E9CAC8E92419F922A2F492D5C0CF
:100E8E00F0E582FD30D50623F582FD181818E685AB
:100E9E0083F084F620D5047B0180027B0308E5F005
:100EAE00D6C6C48583F084C4C6C445F0C48583F019
:100EBE0084D6DBE9E5F024F6500730D10224202455
:100ECE0007243AF70920D509DDC3D0F01818AB82F4
:100EDE0022DDB8181880F3E7F819E7FC19E7FDBD15
:100EEE00FF0122090907B70004190719221919224F
:100EFE00CACDE8C0E0E9C0E0E6FB08E6FA08E6F98C
:100F0E00EFBBFF05120240800A06B6000318060862
:100F1E00120042080618D0E0F9D0E0F8CDCA22E956
:100F2E00FD1BE7B4350FEBFE600709E719F709DE85
:100F3E00F718EDF92240EF09C3E899601AE719B4E2
:100F4E002E04F70980F104B43A067430F70980E7ED
:100F5E00F709E899FE80D1197431F70B80D4286E09
:100F6E00756C6C290049584450434C046C10620057
:100F7E00680023012D022B2020402E80002A091705
:100F8E006F09C578092858092E7309377509F96450
:100F9E0009D66909D6630A0A250A11700AD5660BA5
:100FAE0020650BB3450BAF670C28470C240020209F
:0B0FBE0020204E614E202020464E49AE
:100FC9001200C4EFB2E7FF80031200C4E58124FDDB
:100FD900F8F9E63308E63370060213B60213A504DE
:100FE90060FAEE33EF33700EE6FF18E6FE18E6FD01
:100FF90018E6FC0213B60460E3E58124FBF8D3ECA0
:101009009608ED9608EE9608EFC2E786F0C2F795C6
:10101900F0400FEFC6FF18EEC6FE18EDC6FD18EC3E
:10102900C6FC1213C7C3EB9FF5F0700EE58124FBD4
:10103900F9E4C3CC20D5730211049418605C400E06
:10104900E4FF19E7FE19E7FD19E7FC0210E0E4FFE8
:1010590030F405CEFCE4CDFF30F305E4CECDCCCFA2
:1010690030F21AE5D054184404F8EF54F0D6C4FF0E
:1010790008ECD6C4FC08EDD6C4FDEEC4FE740355D5
:10108900F06012F5F0C3EE13FEED13FDEC13FCEF67
:1010990013FFD5F0F030D55D8009E4CEFFE4FDFC07
:1010A90030D552C3E49FCC191919C797CD09C797F1
:1010B900CE09C797FF4E4D4C70140213B6DB0302DD
:1010C90013A9EC2CFCED33FDEE33FEEF33FFEF30CB
:1010D900E7EBECCFCECDFCEF30E70D0CBC00090DF2
:1010E900BD00050EBE00010BEB7005A2D102139DD8
:1010F900A2D10213B0E42FCC19191937CD0937CE73
:101109000937FF50090BEB700CA2D102139DEFCEEA
:10111900CDCCFF80C2EF13CE13CD13CC13FF80B714
:101129001200C4EF4E601AE58124FEF924FEF8E7A7
:1011390019477019EE33EF33B4FF030213A50213F5
:10114900A9E58124FDF8E63308E63380EB1213C7DD
:10115900248150082B5008A2D502139D2B50DFF78C
:10116900FAE61846197020B7800DEE33CAA2D513D6
:10117900FFCA13FE0213B6EC4D703CBE8046E6FC76
:1011890008E6FD08E680E4EC4D7039BE800280EE89
:10119900E4CEC7CDC6F5F008E4C6CCF9FBFFFA806A
:1011A90076E4CEC9E4CDCAE4FFCCFB803CE4C9CDEA
:1011B900CFCBECCACC8060E4F9FAFBFFCECDCCC52D
:1011C900F00880538CF0E660D8A4C5F0CDFAC5F0DC
:1011D900E6A42DCEF9C5F03400FDE6A42DC5F03402
:1011E90000FDCCFBC5F0CC7F0008E660C0A42EC58D
:1011F900F03C50010DCAFCC5F0CEE6A42AC5F03D6D
:1012090050010FC9FDC5F0CAE6A429C5F03F79010F
:10121900400119CBC5F0CF08E6A42AC5F03F500517
:101229000BBB000109CCC5F0FAE6A42CC5F03B5074
:101239000109CDC5F0CCE6A42DFDC5F039FE330872
:10124900500906B60011A2D502139DEA33FAEC3310
:10125900FCED33FDEE33FEEA30E7140CBC00100D53
:10126900BD000C0EBE000806B60004A2D580D9E662
:05127900A2D50213B034
:10127E00D083D0820213A91200C4EFC2E74E7003CE
:10128E000213A5C082C083E58124FBF8F9E6084667
:10129E0060DE1213C70FBF0006D083D08280E1EF4D
:1012AE0024805007C3CB9B500D80C5CB9B4007D0ED
:1012BE0083D08202139DF6F583EC4D701FBE801C09
:1012CE00E58124FBF8E583A2D513FFE692E7FE182D
:1012DE00E6FD18E6FCD083D0820213B6E58124FB2E
:1012EE00F8E6CEF618E6CDF618E6CCF6EFCCFFE82B
:1012FE002402F9F8E7FA19E7FB19E7FCE4F5F075B3
:10130E00821A758380801DE58303F58330E706A777
:10131E00F009E4F5F0C3EF33FFED33FDEE33FE409D
:10132E000C30E717C3EF9CED9BEE9A400EC3EF9C7B
:10133E00FFED9BFDEE9AFEE58342F0D582C9E7FAFA
:10134E0019E9F81919E720E7191ABA000302127EF3
:10135E00E5F025F0FFE633FC18E633FD18E633FE24
:10136E008009FE09E7FDE6FCE5F0FFEF30E7160C1D
:10137E00BC00120DBD000E0EBE000A0A7007D0830F
:0F138E00D08202139DEAA2D5D083D0820213B081
:10139D0074FF13FF7E80800774FF8001E4FFFEFD64
:1013AD00FC800613FFEE92E7FED0E0F8D0F0E58169
:1013BD0024FCF581C0F0E8C0E022E7D2E7C733098D
:1013CD00E733FB92D592D1EED2E7CE33EF33FF5018
:0413DD0002B2D52261
:1013E1003F8000003DCCCCCD3C23D70A3A83126F1D
:1013F10038D1B7173727C5AC358637BD33D6BF953A
:10140100322BCC7724E69595179ABE150A4FB11F5A
:10141100EB60105407700AEB543803241C12143C7F
:1014210022232312143CEB543870012203241CFBA9
:101431001200ABEB12143C12112C229013E1FC931D
:0E144100FF0CEC93FE0CEC93FD0CEC93FC22E4
:10144F001214958000EC3392D550031214837A2036
:10145F00C3EC20E712EF33FFEE33FEED33FDEC3339
:10146F00FC20E703DAEF22EA247DA2D513FFEC92EA
:10147F00E7CEFC22E4C39FFFE49EFEE49DFDE49CC7
:10148F00FC22C2D580C8EED2E7CE33EF3392D524FB
:10149F0081400CE4C2D5A2D513FC33FDFEFF2224FC
:1014AF00E0500474FF80EFF404FAE4CCCDCECF808B
:1014BF000DC3EF13FFEE13FEED13FDEC13FCDAF18A
:1014CF0020D507EECDFEEFCCFF22E4C39CFCE49DBC
:1014DF00FDE49EFEE49FCCFFEECDFE22EFC2E7FFC0
:1014EF0080A47A083392D5E4FDFEFF30D5031214A1
:1014FF0084EC334010EF33FFEE33FEED33FDEC336E
:10150F00FCDAEE80BEEA247EA2D513CC92E7CDCED4
:03151F00FF80B09A
:10152200E58124FEF88FF063F080E6F96480B5F07F
:101532001B188EF0E6B5F014188DF0E6B5F00D1814
:101542008CF0E6B5F006E4FFFE0213B68FF030F73A
:101552000689F030F701B340077F017E000213B61F
:0715620074FFFFFE0213B647
:101569004241545445525920545950452020202075
:10157900003A4E69434420202020202020202020AA
:1015890020003A4E694D482020202020202020208C
:101599002020003A4C694665202020202020202068
:1015A900202020003A4C69496F202020202020204B
:1015B90020202020003A4C69506F20202020202034
:1015C9002020202020003A534C4120202020202098
:1015D90020202020202000424154544552592043C4
:1015E900454C4C20202020003A4155544F20444579
:1015F9005445435420202020003A253264202020DD
:101609002020202020202020202000424154542E38
:101619002043415041434954592020003A2534641C
:101629006D4168202020202020202000434841527D
:1016390047452043555252454E542020003A2534FF
:10164900646D41202020202020202020003A41558F
:10165900544F2020202020202020202020004449F1
:101669005343482E2043555252454E54202000459D
:1016790058495420424154544552592020202000B1
:101689004E6943442025326443202534646D416802
:10169900004E694D482025326443202534646D414C
:1016A90068004C694665202025316443202534644F
:1016B9006D4168004C69496F20202531644320251C
:1016C90034646D4168004C69506F202025316443B2
:1016D900202534646D416800534C41202020253178
:1016E9006443202534646D416800534554204241C8
:1016F9005454455259205459504500204E69434489
:10170900202020202020202020202000204E694D4C
:1017190048202020202020202020202000204C6943
:101729004665202020202020202020202000204C39
:1017390069496F20202020202020202020200020FF
:101749004C69506F202020202020202020202000BC
:1017590020534C4120202020202020202020202000
:101769000053455420424154544552592043454C55
:101779004C002025326420202020202020202020F9
:101789002020200053455420434150414349545996
:101799002020202000202534646D4168202020204D
:1017A9002020202000202534646D41202020202085
:1017B9002020202000204155544F20202020202087
:1017C9002020202020004C6F6164204D656D6F72D0
:1017D90079205B2532645D0053617665204D656D26
:1017E9006F7279205B2532645D00457261736520F3
:1017F9004D656D6F72795B2532645D004C6F616474
:10180900696E672062617474657279200066726F0F
:101819006D204D656D6F7279205B2532645D002006
:101829004E6F20626174746572792064617461001D
:10183900206174204D656D6F7279205B2532645D7E
:1018490020004F76657277726974652064617461EE
:101859003F200020536176696E6720626174746568
:101869007279200020746F204D656D6F7279205B4D
:101879002532645D2000457261736520646174617D
:101889003F20202020200045726173696E67206225
:1018990061747465727920002045786974204D451A
:1018A9004D4F52592020202000204E6943442025C5
:1018B900326443202534646D416800204E694D48E7
:1018C9002025326443202534646D416800204C6929
:1018D9004665202025316443202534646D41680024
:1018E900204C69496F202025316443202534646DDB
:1018F900416800204C69506F202025316443202520
:1019090034646D41680020534C4120202025316406
:1019190043202534646D41680020456D7074792039
:101929004D656D6F72792020200020202020202015
:10193900202020202020202020200045726173656E
:1019490020616C6C20646174613F20004572617391
:10195900696E6720616C6C206461746100202020CD
:0E19690066726F6D204D656D6F7279202000E3
:101977005345542043454C4C532044455445435408
:1019870000204D414E55414C202020202020202072
:1019970020005345542043484152474552204D4F5C
:1019A700444500204359434C45204348415247454D
:1019B7002020200020434841524745204F4E4C5994
:1019C70020202020002044495343484152474520C6
:1019D7004F4E4C59200053455420434841524745E8
:1019E700204359434C450053455420534F554E44CB
:1019F70020564F4C554D4500204F4E20202020208B
:101A0700202020202020202000204F464620202074
:101A170020202020202020202000534554205452ED
:101A27004947474C45204D4F44450020202A2A204E
:101A37004552524F52202A2A2020200020204D654F
:101A47006D6F7279204661696C20202000204C4F11
:101A57004144202020202053415645202000205378
:101A67004156452020202020455241534520002043
:101A7700455241534520202020464F524D415400A6
:101A870020464F524D41542020204558495420208C
:101A970000204558495420202020204C4F41442005
:101AA7002000557365203C3E20746F2053656C659C
:101AB700637400204E6F74204170706C69636162BB
:101AC7006C652000466F7220546869732042617408
:101AD700746572790020466F722054686973204DCF
:101AE7006F64652020002043454C4C5320444554E7
:101AF700454354494F4E003A4D414E55414C2020E5
:101B070020202020202020002043484152474552D2
:101B1700204D4F4445202020003A4359434C45204F
:101B2700434841524745202020003A434841524705
:101B370045204F4E4C5920202020003A444953431A
:101B47004841524745204F4E4C59200020434841B9
:101B5700524745204359434C45202020003A4E6FB9
:101B670074204170706C696361626C65200020535A
:101B77004F554E4420564F4C554D45202020003A96
:101B87004F4E202020202020202020202020200011
:101B97003A4F4646202020202020202020202020A9
:101BA700002054524947474C45204D4F444520207B
:101BB70020002045584954204F5054494F4E532038
:101BC700202000204241545445525920204D454D74
:101BD7004F525900204D454D4F525920204F5054D8
:101BE700494F4E5300204F5054494F4E5320202009
:101BF7002045584954002045584954202020204268
:101C0700415454455259002020534D4152542043CA
:101C170048415247455220002020534552564943D8
:101C270045204D4F44452020002020202046495282
:101C37004D57415245202020200020205645525321
:101C4700494F4E20312E31386120002044495343FB
:101C57004820432D53544550202020003A25346412
:101C67002020202020202020202020002043555203
:101C770052454E54205354455020202000205354A1
:101C87004152542044454C415920202020003A25F8
:101C97003364205365636F6E647320202020002017
:101CA70044495343482D4348472044454C41590034
:101CB700204D41582E20564F4C542F43454C4C2015
:101CC700003A25352E32665620202020202020205D
:101CD7002020003A44495341424C452020202020EF
:101CE70020202000204D494E2E20564F4C542F4384
:101CF700454C4C2000204E6943442053454E5349E0
:101D07005449564520003A253264206D562F4365C5
:101D17006C6C20202020202000205043204C494E6E
:101D27004B2020202020202020003A454E41424CC5
:101D370045202020202020202020002053555050CF
:101D47004C59204D4F4E49544F5220003A43482595
:101D570031642020202025352E326656732000203E
:101D6700564F4C544147452053544550202020009E
:101D77003A2534642020202025352E32665620004F
:101D8700205741544348444F472054494D4552201A
:101D97000020455849542053455256494345202071
:101DA700200053455420444953434820432D53545E
:101DB7004550005345542043555252454E542053E5
:101DC70054455000534554205354415254204445E0
:101DD7004C415920005345542044495343482D430F
:101DE700484152474500534554204D41582E2056EF
:101DF7002F43454C4C20003A25352E32665620207D
:101E07002020202020202000534554204D494E2ECD
:101E170020562F43454C4C20004E694344205345E0
:101E27004E5349544956452020003A253264206DC7
:101E370056202020202020202020200053455420F9
:101E47005043204C494E4B20202020200020454E57
:101E570041424C45202020202020202020002044E3
:101E6700495341424C452020202020202020005368
:101E7700455420535550504C59204D4F4E2E20005D
:101E870053455420564F4C544147452053544550D1
:101E970000534554205741544348444F472020207E
:021EA700200019
:071EA9007803EFF21207F5C8
:101EB0009000DEE0B403028074500CE06017146000
:101EC0001414603F021F7FE024FC60611470030261
:051ED0001F56021F7FF8
:101ED5009000DF7405F0A37478F07401900116F09A
:101EE500740C7904F37905740FF30974A0F3790779
:101EF5007407F30974D0F374017909F3807C9000B9
:101F0500DF740EF0A37410F07402900116F07404DF
:101F15007904F37905740FF30974A0F37907E4F3F1
:101F250009F3047909F380529000DF7410F0A3746B
:101F350068F07402900116F0047904F37905740FC2
:101F4500F30974A0F37907E4F309F3047909F3803D
:101F5500299000DF7409F0A37492F07402900116C1
:101F6500F074067904F37905741BF3097458F37951
:101F750007E4F309F374037909F3129672EF790A0A
:101F8500F3E3B40403E3FF227903E314601B147045
:101F9500030223BE14700302243B1470030226417E
:091FA5001470030227A1021EB012
:101FAE007F017B057A1679F31295A9790AE3B401BC
:011FBE00150D
:101FBF009000DEE0B40001D34005E014F080067419
:101FCF00059000DEF0790AE3B402028003022309D0
:101FDF009000DEE0FAB403028056500CEA6014144D
:101FEF0060251460350220ABEA24FC604314607650
:031FFF000220AB12
:102002009000D37403F0A374E8F09000DAE4F0A334
:10201200F00220AB9000D37407F0A304F09000DA32
:10202200E4F0A3F00220AB9000D37408F0A374FC98
:10203200F09000DA740BF0A374B8F0806C9000D3C7
:102042007408F0A374FCF0E4FCFD9000D3E0FEA35E
:10205200E0FF121491C004C005C006C0077433FE2D
:10206200FCFD743FFF12112C121495EE9000DAF071
:10207200A3EFF09000D37405F0A37414F0E4FCFD18
:102082009000D3E0FEA3E0FF121491C004C005C08B
:1020920006C007E4FCFD7440FE14FF12112C12145A
:1020A20095EE9000DAF0A3EFF09000DEE0B40101CB
:1020B200D340179000DAE0B40005A3E0B464005006
:1020C200099000DAE4F0A37464F09000DAE0FEA371
:1020D200E0FFE4FC7D64120179EE9000DAF0A3EFF8
:1020E200F09000DAE0FEA3E0FFE4FC7D6412013D23
:1020F200EE9000DAF0A3EFF0BE0B04BFB801D340BC
:102102000A9000DA740BF0A374B8F09000D3E0F5F3
:10211200F0A3E0FB7905E3B5F00509E3B503005050
:102122000B79059000D3E3F009A3E3F07F05129C3D
:10213200BAEE790BF309EFF3E4FCFD90011EE0FE29
:10214200A3E0FF121491C004C005C006C00774CDFD
:10215200FC14FDFE743DFF12112C790D1200F4E403
:10216200FCFD790BE3FE09E3FF121491C004C005E4
:10217200C006C007780D1200DC121288C004C00528
:10218200C006C0077466FEFCFD743FFF121522BF35
:07219200010280030222FCA0
:102199009000DEE0B40303022260500CE0601A14E0
:1021A90060171460630222FAE024FC7003022260C3
:0921B9001470030222AE0223039C
:1021C200E4FCFD790BE3FE09E3FF121491C004C0A5
:1021D20005C006C007780D1200DC121288C004C0C8
:1021E20005C006C0077CF57DBE7E207F4012112C03
:1021F200C004C005C006C00774ABFC14FDFE743EEB
:10220200FF12112C121495EF9000D5F0022303E473
:10221200FCFD790BE3FE09E3FF121491C004C00533
:10222200C006C007780D1200DC121288C004C00577
:10223200C006C0077CB07DDE7E687F3F12112CC0D5
:1022420004C005C006C00774ABFC14FDFE743EFF5B
:1022520012112C121495EF9000D5F0022303E4FC26
:10226200FD790BE3FE09E3FF121491C004C005C01F
:1022720006C007780D1200DC121288C004C005C027
:1022820006C0077C737D717E557F3F12112CC004FE
:10229200C005C006C00774ABFC14FDFE743EFF12FD
:1022A200112C121495EF9000D5F08055E4FCFD79C5
:1022B2000BE3FE09E3FF121491C004C005C006C07F
:1022C20007780D1200DC121288C004C005C006C0D7
:1022D200077C207D527EC07F3F12112CC004C005B6
:1022E200C006C00774ABFC14FDFE743EFF12112C35
:0A22F200121495EF9000D5F080075C
:1022FC007909E39000D5F012965FE4FF22790AE3A6
:03230C00B4031304
:10230F009000DEE0B405005005E004F08005E49095
:10231F0000DEF09000DEE0700F7B027A0079E17D45
:10232F00057C17780412081D9000DEE0FAB4010F47
:10233F007B027A0079E17D057C17781512081D90D4
:10234F0000DEE0FAB4020F7B027A0079E17D057CB2
:10235F0017782612081D9000DEE0FAB4030F7B02F7
:10236F007A0079E17D057C17783712081D9000DE21
:10237F00E0FAB4040F7B027A0079E17D057C1778CF
:10238F004812081D9000DEE0FAB4050F7B027A00B8
:10239F0079E17D057C17785912081D74069000E1CC
:1023AF00F07F027B027A0079E11295A9021EB07FBD
:1023BF00017B057A17796A1295A9790AE3B4011599
:1023CF007909E3F5F09000D5E0B5F001D340069020
:0B23DF0000D5E014F0790AE3B4020618
:1023EA0012965FE4FF22790AE3B403147904E3F551
:1023FA00F09000D5E0B5F00050069000D5E004F06A
:10240A009000D5E0FBE4C0E0C0037B027A0079E1EA
:10241A007D057C17787B12081D158115817406903D
:10242A0000E1F07F027B027A0079E11295A9021E8F
:10243A00B07F017B057A17798D1295A99000D3E0B8
:10244A00FAA3E0BA0003B4640050099000D3E4F0A0
:10245A00A37464F09000D3E0F5F0A3E0FB7905E300
:10246A00B5F00509E3B50300500B79059000D3E3F5
:10247A00F009A3E3F0790AE3B401209000D3E0B4B1
:10248A000006A3E0B46401D340119000D4E024CE46
:10249A00FB9000D3E034FFF0A3EBF0790AE3B40237
:0624AA000280030225E29E
:1024B0009000DEE06004E0B401079000DAE4F0A3ED
:1024C000F09000DEE0FAB402309000D3E0FAA3E02E
:1024D000FBE4FCFDAE02AF03121491C004C005C0C2
:1024E00006C0077C147DAE7EA77F3F12112C12140C
:1024F00095EE9000DAF0A3EFF09000DEE0FA6403CE
:102500006003BA042C9000D3E0FEA3E0FFE4FCFDDE
:10251000121491C004C005C006C0077433FEFCFD50
:10252000743FFF12112C121495EE9000DAF0A3EF15
:10253000F09000DEE0B4052C9000D3E0FEA3E0FFB5
:10254000E4FCFD121491C004C005C006C007E4FC01
:10255000FD7440FE14FF12112C121495EE9000DA57
:10256000F0A3EFF09000DEE0FAB40101D340179041
:1025700000DAE0B40005A3E0B4640050099000DA8A
:10258000E4F0A37464F0E4FCFD9000DAE0FEA3E064
:10259000FF121491C004C005C006C0077C0A7DD795
:1025A0007E237F3C12112C121495EE9000DAF0A3DA
:1025B000EFF09000DAE0FEA3E0FFE4FC7D6412019E
:1025C0003DEE9000DAF0A3EFF0BE0B04BFB801D3EC
:1025D000400A9000DA740BF0A374B8F012965FE42E
:1025E000FF22790AE3B403289000D37905E3F5F0DC
:1025F000E0B5F00909E3F5F0A3E0B5F00050119063
:1026000000D4E02432FB9000D3E03400F0A3EBF0E0
:102610009000D3E0C0E0A3E0C0E07B027A0079E163
:102620007D057C17789E12081D1581158174069012
:1026300000E1F07F027B027A0079E11295A9021E87
:10264000B07F017B057A1679351295A99000DEE0FE
:10265000FAB40101D340179000DAE0B40005A3E01A
:10266000B4640050099000DAE4F0A37464F09000C0
:10267000DAE0FAA3E0BA0B04B4B801D3400A900040
:10268000DA740BF0A374B8F09000DEE0B40101D36B
:02269000406B9D
:10269200790AE3B4010280030227239000DAE0B44E
:1026A2000006A3E0B46401D34077E4FCFD9000DAB5
:1026B200E0FEA3E0FF121491C004C005C006C007EB
:1026C2009000D3E4FCFDE0FEA3E0FF121491C004ED
:1026D200C005C006C00774CDFC14FDFE743DFF1298
:1026E200112C121522BF01399000DBE0249CFB90D3
:0B26F20000DAE034FFF0A3EBF08026DC
:1026FD00790AE3B401209000DAE0B40006A3E0B457
:10270D000001D340119000DBE0249CFB9000DAE047
:0C271D0034FFF0A3EBF0790AE3B40206ED
:1027290012965FE4FF22790AE3B4031F9000DAE00E
:10273900B40B05A3E0B4B80050119000DBE02464A9
:10274900FB9000DAE03400F0A3EBF09000DAE0FA55
:10275900A3E0FBBA0004B40001D34019C002C003CE
:102769007B027A0079E17D057C1778AE12081D1588
:10277900811581800F7B027A0079E17D057C1778CC
:10278900BE12081D74069000E1F07F027B027A00F8
:1027990079E11295A9021EB07F017B057A16796746
:1027A9001295A99000DCE0FAA3E0BA0003B4640032
:1027B90050099000DCE4F0A37464F0790AE3B401F1
:1027C900209000DCE0B40006A3E0B46401D340111A
:1027D9009000DDE0249CFB9000DCE034FFF0A3EBEB
:0727E900F0790AE3B40206D7
:1027F00012965FE4FF22790AE3B403287907E3F530
:10280000F09000DCE0B5F00909E3F5F0A3E0B5F0E5
:102810000050119000DDE02464FB9000DCE0340007
:10282000F0A3EBF09000DCE0C0E0A3E0C0E07B02AE
:102830007A0079E17D057C1778AE12081D158115A7
:102840008174069000E1F07F027B027A0079E11248
:0528500095A9021EB075
:102855007811EFF27912E4F30904F37914E4F3093A
:102865007410F319E3FE09E3FF129A78EE7916F373
:1028750009EFF37915E32401FF19E33400FE129AF9
:1028850078EF9000AFF07915E32402FF19E33400E7
:10289500FE129A78EE9000A4F0A3EFF07915E324E8
:1028A50003FF19E33400FE129A78EF9000A6F012A8
:0228B50007F525
:1028B700129672EF7918F37911E314600E14600B16
:0B28C70014600814700302327080E5FA
:1028D2007911E3B4011C7912E3C0E009E3C0E07BA3
:1028E200027A0079E17D057C1778CF12081D1581E7
:1028F20015817911E3B4021C7912E3C0E009E3C047
:10290200E07B027A0079E17D057C1778E112081DEF
:10291200158115817911E3B4031C7912E3C0E00932
:10292200E3C0E07B027A0079E17D057C1778F3123F
:10293200081D158115817918E3B40102800302296B
:10294200E27912E3B4000609E3B40001D3500302B2
:0229520029E278
:102954007913E314F3F4197003E314F37912E3B471
:0A296400000609E3B40001D3406C43
:10296E007913E324FFFF19E334FFFEE4FC7D0A1222
:10297E00013DEF2410FFE43E7914F309EFF319E360
:10298E00FE09E3FF129A78EE7916F309EFF3791543
:10299E00E32401FF19E33400FE129A78EF9000AFA2
:1029AE00F07915E32402FF19E33400FE129A78EE53
:1029BE009000A4F0A3EFF07915E32403FF19E3349C
:0C29CE0000FE129A78EF9000A6F080083E
:1029DA007912E4F309740BF37918E3B40202800361
:0329EA00022FF3C6
:1029ED007912E3B4000809E3B40B03E4FF22791173
:0929FD00E3B401028003022B5F28
:102A06007813E22400FB18E23455F5F07916E3B5A5
:102A1600F0028003022B1609E3B503028003022BA2
:012A26001699
:102A27007F017B057A1879051295A97912E3C0E031
:102A370009E3C0E07B027A0079E17D057C1878160E
:102A470012081D158115817F027B027A0079E11238
:102A570095A97913E324FFFF19E334FFFEE4FC7D16
:102A67000A12013DEF2410FFE43E7914F309EFF356
:102A7700E32401FF19E33400FE129A78EF9000DE99
:102A8700F07915E32402FF19E33400FE129A78EE79
:102A97009000D3F0A3EFF07915E32403FF19E33493
:102AA70000FE129A78EF9000D5F07915E32404FF21
:102AB70019E33400FE129A78EE9000DAF0A3EFF0F3
:102AC7007915E32405FF19E33400FE129A78EE9096
:102AD70000DCF0A3EFF07915E32406FF19E33400D7
:102AE700FE129A78EE9000DFF0A3EFF0129B09E454
:102AF700FE7F0E129B62E4FE7F0E7912E3FC09E370
:0F2B0700FD129A3F129B8A12965FD208E4FF22BA
:102B160012965F7F017B057A1879281295A979129A
:102B2600E3C0E009E3C0E07B027A0079E17D057C41
:102B360018783912081D158115817F027B027A00EB
:102B460079E11295A9E4FE7F6412964712965F7E9C
:102B5600057FDC129647E4FF227911E3B402028076
:042B660003022E0830
:102B6A007813E22400FB18E23455F5F07916E3B540
:102B7A00F0028003022D0109E3B503028003022D4E
:012B8A000149
:102B8B007B057A18794B129308EF64016003022ED0
:012B9B000831
:102B9C007F017B057A18795C1295A97912E3C0E064
:102BAC0009E3C0E07B027A0079E17D057C18786D41
:102BBC0012081D158115817F027B027A0079E112C2
:102BCC0095A9129B097913E324FFFF19E334FFFE47
:102BDC00E4FC7D0A12013DEF2410FFE43E7914F36E
:102BEC0009EFF319E3FE09E3FF129B627915E32465
:102BFC0001FF19E33400FE129B627915E32402FFF6
:102C0C0019E33400FE129B627915E32403FF19E3E8
:102C1C003400FE129B627915E32404FF19E334009F
:102C2C00FE129B627915E32405FF19E33400FE12B2
:102C3C009B627915E32406FF19E33400FE129B62B4
:102C4C007914E3FE09E3FF7813E22400FD18E23463
:102C5C0055FC129A3F7915E32401FF19E33400FE69
:102C6C009000DEE0FD7C00129A3F7915E32402FF10
:102C7C0019E33400FE9000D3E0FCA3E0FD129A3F70
:102C8C007915E32403FF19E33400FE9000D5E0FD31
:102C9C007C00129A3F7915E32404FF19E33400FEFB
:102CAC009000DAE0FCA3E0FD129A3F7915E32405CD
:102CBC00FF19E33400FE9000DCE0FCA3E0FD129A67
:102CCC003F7915E32406FF19E33400FE9000DFE0A2
:102CDC00FCA3E0FD129A3FE4FE7F0E129B62E4FE21
:102CEC007F0E7912E3FC09E3FD129A3F129B8A12C4
:052CFC00965FE4FF22D9
:102D01007F017B057A18795C1295A97912E3C0E0FD
:102D110009E3C0E07B027A0079E17D057C18786DDA
:102D210012081D158115817F027B027A0079E1125B
:102D310095A9129B097913E324FFFF19E334FFFEE0
:102D4100E4FC7D0A12013DEF2410FFE43E7914F307
:102D510009EFF319E3FE09E3FF7913E32400FD19F9
:102D6100E33455FC129A3F7915E32401FF19E3344A
:102D710000FE9000DEE0FD7C00129A3F7915E3240D
:102D810002FF19E33400FE9000D3E0FCA3E0FD1242
:102D91009A3F7915E32403FF19E33400FE9000D52F
:102DA100E0FD7C00129A3F7915E32404FF19E33416
:102DB10000FE9000DAE0FCA3E0FD129A3F7915E3F2
:102DC1002405FF19E33400FE9000DCE0FCA3E0FDE4
:102DD100129A3F7915E32406FF19E33400FE9000AF
:102DE100DFE0FCA3E0FD129A3FE4FE7F0E129B623E
:102DF100E4FE7F0E7912E3FC09E3FD129A3F129B78
:102E01008A12965FE4FF227911E3B4030280030280
:022E11002FF39D
:102E13007813E22400FB18E23455F5F07916E3B594
:102E2300F0028003022F1C09E3B503028003022F83
:012E33001C82
:102E34007B057A18797F129308EF64016003022FEF
:012E4400F39A
:102E45007F017B057A1879901295A97912E3C0E084
:102E550009E3C0E07B027A0079E17D057C187816EC
:102E650012081D158115817F027B027A0079E11216
:102E750095A9129B097913E324FFFF19E334FFFE9B
:102E8500E4FC7D0A12013DEF2410FFE43E7914F3C2
:102E950009EFF319E3FE09E3FF129B627915E324B9
:102EA50001FF19E33400FE129B627915E32402FF4A
:102EB50019E33400FE129B627915E32403FF19E33D
:102EC5003400FE129B627915E32404FF19E33400F4
:102ED500FE129B627915E32405FF19E33400FE1207
:102EE5009B627915E32406FF19E33400FE129B6209
:102EF5007915E32407FF19E33400FE129B62E4FE13
:102F05007F0E129B62E4FDFEFC7F0E129A3F129B20
:072F15008A12965FE4FF221F
:102F1C007F017B057A1879901295A97912E3C0E0AC
:102F2C0009E3C0E07B027A0079E17D057C18781614
:102F3C0012081D158115817F027B027A0079E1123E
:102F4C0095A9129B097913E324FFFF19E334FFFEC3
:102F5C00E4FC7D0A12013DEF2410FFE43E7914F3EA
:102F6C0009EFF319E3FE09E3FF129B627915E324E1
:102F7C0001FF19E33400FE129B627915E32402FF72
:102F8C0019E33400FE129B627915E32403FF19E365
:102F9C003400FE129B627915E32404FF19E334001C
:102FAC00FE129B627915E32405FF19E33400FE122F
:102FBC009B627915E32406FF19E33400FE129B6231
:102FCC007915E32407FF19E33400FE129B62E4FE3B
:102FDC007F0E129B62E4FDFEFC7F0E129A3F129B49
:102FEC008A12965FE4FF227918E3B403028003028D
:102FFC0030A27912E3B4000509E3B40C00400302DB
:02300C0030A2F0
:10300E007913E304F3197003E304F37912E3B400C4
:10301E000C09E3B40C077912E4F30904F37912E313
:0A302E00B4000509E3B40B00506A7A
:103038007913E324FFFF19E334FFFEE4FC7D0A1251
:10304800013DEF2410FFE43E7914F309EFF319E38F
:10305800FE09E3FF129A78EE7916F309EFF3791572
:10306800E32401FF19E33400FE129A78EF9000AFD1
:10307800F07915E32402FF19E33400FE129A78EE82
:103088009000A4F0A3EFF07915E32403FF19E334CB
:1030980000FE129A78EF9000A6F07912E3B4001AB5
:0530A80009E3B40B1563
:1030AD007B027A0079E17D057C1878A112081D74E8
:1030BD00069000E1F07F017B027A0079E11295A97B
:1030CD007918E3B404037F04227813E22400FB187B
:1030DD00E23455F5F07916E3B5F002800302323291
:0A30ED0009E3B5030280030232324A
:1030F7009000AFE0B4030302319E500CE0601A1455
:103107006041146068023217E024FC70030231C783
:093117001470030231F0023217BA
:103120009000A4E0C0E0A3E0C0E0A3E0FBE4C0E0C6
:10313000C0037B027A0079E17D057C1878B2120821
:103140001D74FC2581F5810232179000A4E0C0E0D7
:10315000A3E0C0E0A3E0FBE4C0E0C0037B027A0090
:1031600079E17D057C1878C412081D74FC2581F571
:10317000810232179000A4E0C0E0A3E0C0E0A3E029
:10318000FBE4C0E0C0037B027A0079E17D057C1896
:1031900078D612081D74FC2581F581023217900043
:1031A000A4E0C0E0A3E0C0E0A3E0FBE4C0E0C00313
:1031B0007B027A0079E17D057C1878E912081D749C
:1031C000FC2581F58180509000A4E0C0E0A3E0C020
:1031D000E0A3E0FBE4C0E0C0037B027A0079E17D7C
:1031E000057C1878FC12081D74FC2581F581802768
:1031F0009000A4E0C0E0A3E0C0E0A3E0FBE4C0E0F6
:10320000C0037B027A0079E17D057C19780F1208F2
:103210001D74FC2581F5819000D5E0600790010CBC
:04322000E0B4011DF8
:0E32240074209000E7F074419000E8F0800FF5
:103232007B027A0079E17D057C19782212081D74DF
:10324200069000E1F07912E3B4000509E3B40B0043
:10325200500E7F027B027A0079E11295A90233AC0B
:103262007F027B057A1979331295A90228B77B056B
:0F3272007A197944129308EF640160030233ACB8
:103281007F017B057A1979551295A97F027B057A11
:103291001979661295A9129B09129B1FE4FE7F649E
:1032A100129647E4FDFEFF7C01129A3FE4FE7F0186
:1032B10090010CE0FD7C00129A3F900116E0FBE4C6
:1032C1007914F309EBF3900119E0B4010C7915E3DA
:1032D1004480FB19E3F309EBF390011BE0B4010C0B
:1032E1007915E34440FB19E3F309EBF3E4FE7F02B4
:1032F1007914E3FC09E3FD129A3FE4FE7F03900198
:103301001CE0FD7C00129A3FE4FE7F0490011DE069
:10331100FD7C00129A3FE4FE7F05900113E0FCA3BF
:10332100E0FD129A3FE4FE7F06900109E0FCA3E074
:10333100FD129A3FE4FE7F0790011EE0FCA3E0FD31
:10334100129A3FE4FE7F08900110E0FCA3E0FD1219
:103351009A3FE4FE7F09900117E0FD7C00129A3F3D
:10336100E4FE7F0A900120E0FD7C00129A3FE4FE1A
:103371007F0B90011AE0FD7C00129A3FE4FE7F0C66
:1033810090010DE0FD7C00129A3FE4FE7F0D90015B
:103391000EE0FCA3E0FD129A3FE4FDFEFC7F0E125D
:0E33A1009A3F129B8A12965FE4FF220228B721
:0733AF007819EFF21207F597
:1033B600129672EF791AF3E3B404037F04227919A3
:1033C600E314601A14700302347614700302353A5B
:0E33D6001470030235B514700302364780D21E
:1033E4007F017B057A1979771295A990010CE0B4D5
:1033F40001117B027A0079E17D057C1778BE120801
:103404001D800F7B027A0079E17D057C1978881292
:10341400081D74069000E1F07F027B027A0079E1D6
:0E3424001295A9791AE364016004E3B4031160
:1034320090010CE0B40104E4F08006740190010CE8
:0C344200F0791AE3B4020280030236F8AD
:07344E00900115E0B4011B21
:10345500129B09E4FE7F01129B62E4FE7F0190014D
:103465000CE0FD7C00129A3F129B8A12965FE4FFE6
:10347500227F017B057A1979991295A9791AE3B406
:0234850001152F
:10348700900116E0B40101D34005E014F080067402
:0B34970003900116F0791AE3B402283C
:0734A200900115E0B4011BCD
:1034A900129B09E4FE7F02129B62E4FE7F029001F7
:1034B90016E0FD7C00129A3F129B8A12965FE4FF88
:0734C90022791AE3B4031499
:1034D000900116E0B403005005E004F0800674018A
:1034E000900116F0900116E0B4010F7B027A00798A
:1034F000E17D057C1978AA12081D900116E0B4023E
:103500000F7B027A0079E17D057C1978BB12081DDA
:10351000900116E0B4030F7B027A0079E17D057C0F
:103520001978CC12081D74069000E1F07F027B022E
:103530007A0079E11295A90233B67F017B057A19E9
:1035400079DD1295A990010BE0FBE4C0E0C0037B9C
:10355000027A0079E17D057C16780212081D15813A
:10356000158174069000E1F07F027B027A0079E118
:103570001295A9791AE3B4011090010BE0B401018E
:0F358000D3400690010BE014F0791AE3B4020671
:10358F0012965FE4FF22791AE3B403028003023636
:10359F00F890010BE0B40A0040030236F890010BDB
:1035AF00E004F00233B67F017B057A1979EE1295AC
:1035BF00A990011CE0B401117B027A0079E17D052D
:1035CF007C1978FF12081D800F7B027A0079E17D4C
:1035DF00057C1A781012081D74069000E1F07F0226
:1035EF007B027A0079E11295A9791AE364016004EC
:0435FF00E3B403111D
:1036030090011CE0B40104E4F08006740190011CF5
:0C361300F0791AE3B4020280030236F8DA
:07361F00900115E0B4011B4E
:10362600129B09E4FE7F03129B62E4FE7F03900176
:103636001CE0FD7C00129A3F129B8A12965FE4FF03
:10364600227F017B057A1A79211295A990011BE048
:10365600B401117B027A0079E17D057C1978FF12AD
:10366600081D800F7B027A0079E17D057C1A7810AF
:1036760012081D74069000E1F07F027B027A007941
:0F368600E11295A9791AE364016004E3B403111A
:1036950090011BE0B40104E4F08006740190011B65
:0736A500F0791AE3B4024CB6
:0736AC00900115E0B4013F9D
:1036B300900116E0791BF3900119E0B40108791B1E
:1036C300E34480791BF390011BE0B40108791BE309
:1036D3004440791BF3129B09E4FE7F02129B62E4D0
:1036E300FE7F02791BE3FD7C00129A3F129B8A1234
:0836F300965FE4FF220233B6EA
:0836FB007401791FF31207F5B9
:10370300129672EF7920F3E3146012146028147098
:0D371300030237C21470030237D80237DBFF
:10372000791FE3B40101D34008791FE314F3023792
:0F373000DB7406791FF30237DB791FE3B406065B
:06373F001207F5E4FF2271
:10374500791FE364026009E364036004E3B40529B7
:0A3755009000DEE0B40101D3401F34
:10375F007F017B057A1A79BA1295A97F027B057AC8
:10376F001A79CB1295A97E077FD0129647803F79A1
:0D377F001FE3B40327900116E06401601FF2
:10378C007F017B057A1A79BA1295A97F027B057A9B
:0F379C001A79DC1295A97E077FD012964780120A
:1037AB00791FE3FF1233AFEF7821F2E2B404037F0A
:1037BB0004221207F58019791FE3B406005007792C
:1037CB001FE304F3800A7401791FF380037F042243
:1037DB00791FE3B404030239165010E314601D146F
:1037EB00605D1470030238A80239D0E324FB700328
:0C37FB000239591470030239A50237038B
:103807007B027A0079E17D057C1A78ED12081D7438
:10381700069000E1F07F017B027A0079E11295A919
:1038270090010CE0B4010E7F027B057A16795612DF
:1038370095A90239D07F027B057A1A79FE1295A9DC
:103847000237037B027A0079E17D057C1B780F1232
:10385700081D74069000E1F07F017B027A0079E190
:103867001295A9900116E0B4010B7F027B057A1B24
:1038770079201295A9900116E0B4020B7F027B050F
:103887007A1B79311295A9900116E0B403028003DF
:103897000239D07F027B057A1B79421295A902373C
:1038A700037B027A0079E17D057C1B785312081DA2
:1038B70074069000E1F07F017B027A0079E11295AE
:1038C700A99000DEE0B40101D35008900116E0642E
:1038D7000160117B027A0079E17D057C1B78641217
:1038E700081D801D90010BE0FBE4C0E0C0037B02D4
:1038F7007A0079E17D057C16780212081D1581157D
:10390700817F027B027A0079E11295A90237037B56
:10391700027A0079E17D057C1B787512081D740613
:103927009000E1F07F017B027A0079E11295A9907E
:10393700011CE0B4010E7F027B057A1B7986129584
:10394700A90239D07F027B057A1B79971295A902C4
:1039570037037B027A0079E17D057C1B78A8120882
:103967001D74069000E1F07F017B027A0079E11275
:1039770095A990011BE0B401179000DEE0B40101A6
:10398700D3500D7F027B057A1B79861295A9803962
:103997007F027B057A1B79971295A90237037B0271
:1039A7007A0079E17D057C1B78B912081D740690B1
:1039B70000E1F07F017B027A0079E11295A97F028D
:0C39C7007B057A1979331295A9023703A9
:0739D300E47922F31207F56D
:1039DA00129672EF7923F3E314600C1460221470C8
:0739EA0003023A8B023A9E32
:1039F1007922E3B40001D340087922E314F3023AB7
:103A01009E74037922F3023A9E7922E3600C1460DA
:0A3A11002B14604E14606D023A9E03
:103A1B00120271EF7924F31207F57924E3B4045EF3
:103A2B0012965F308003208155E4FE7F6412964727
:103A3B0080F1120695EF7924F31207F57924E3B49C
:023A4B00041263
:103A4D0012965F308003208109E4FE7F6412964751
:103A5D0080F1300827221236FBEF7924F31207F597
:063A6D007924E3B4041605
:103A730012965F30800320810DE4FE7F6412964727
:103A830080F11207F52280137922E3B40300500773
:103A93007922E304F38004E47922F37922E3600BCF
:0B3AA300146019146027146035804285
:103AAE007B027A0079E17D057C1B78CA12081D80A5
:103ABE00317B027A0079E17D057C1B78DB12081DD3
:103ACE0080207B027A0079E17D057C1B78EC120860
:103ADE001D800F7B027A0079E17D057C1B78FD123B
:103AEE00081D74069000E1F07F017B027A0079E1F7
:103AFE001295A97B027A0079E17D057C1A78A912CC
:103B0E00081D74059000E5F0049000E6F07F027B3E
:0B3B1E00027A0079E11295A90239DA61
:103B29007F017B057A1C790E1295A97F027B057AA4
:103B39001C791F1295A97E057FDC1296477F017BB0
:103B4900057A1C79301295A97F027B057A1C794187
:103B59001295A97E057FDC129647E47925F31207B1
:013B6900F566
:103B6A00129672EF7926F3E314600814601C14604D
:033B7A002F804059
:103B7D007925E3B40001D340077925E314F38030B0
:0D3B8D00740B7925F380297925E3B40B042E
:043B9A001207F522F7
:103B9E007925E3FF1240471207F580137925E3B428
:103BAE000B0050077925E304F38004E47925F379BB
:103BBE0025E3B40C004003024044FA232A903BCF85
:103BCE0073023BF6023C41023C8C023CD7023D2282
:103BDE00023DAC023E18023E63023EA6023F400288
:083BEE003FD7024019023B6AB7
:103BF6007B027A0079E17D057C1C785212081D74DF
:103C0600069000E1F07F017B027A0079E11295A926
:103C160090010EE0C0E0A3E0C0E07B027A0079E10B
:103C26007D057C1C786312081D158115817F027B3A
:103C3600027A0079E11295A9023B6A7B027A007941
:103C4600E17D057C1C787312081D74069000E1F076
:103C56007F017B027A0079E11295A9900109E0C003
:103C6600E0A3E0C0E07B027A0079E17D057C1C7868
:103C76006312081D158115817F027B027A0079E1A6
:103C86001295A9023B6A7B027A0079E17D057C1CCC
:103C9600788412081D74069000E1F07F017B027A99
:103CA6000079E11295A990011AE0FBE4C0E0C00397
:103CB6007B027A0079E17D057C1C789512081D153A
:103CC6008115817F027B027A0079E11295A9023B78
:103CD6006A7B027A0079E17D057C1C78A612081DB4
:103CE60074069000E1F07F017B027A0079E112957B
:103CF600A990010DE0FBE4C0E0C0037B027A0079E5
:103D0600E17D057C1C789512081D158115817F02C1
:103D16007B027A0079E11295A9023B6A7B027A005E
:103D260079E17D057C1C78B712081D74069000E1C8
:103D3600F07F017B027A0079E11295A9900113E0E8
:103D4600FAA3E0FBBA0704B46C01D3503CE4FCFDD3
:103D5600AE02AF03121491C004C005C006C0077CB2
:103D66006F7D127E837F3A12112CC004C005C006F7
:103D7600C0077B027A0079E17D057C1C78C81208B1
:103D86001D74FC2581F581800F7B027A0079E17D27
:103D9600057C1C78DA12081D7F027B027A0079E125
:103DA6001295A9023B6A7B027A0079E17D057C1CAB
:103DB60078EB12081D74069000E1F07F017B027A11
:103DC6000079E11295A9E4FCFD900110E0FEA3E064
:103DD600FF121491C004C005C006C0077C6F7D1297
:103DE6007E837F3A12112CC004C005C006C0077B33
:103DF600027A0079E17D057C1C78C812081D74FCE6
:103E06002581F5817F027B027A0079E11295A9026C
:103E16003B6A7B027A0079E17D057C1C78FC1208FE
:063E26001D74069000E18E
:103E2C00F07F017B027A0079E11295A9900117E0ED
:103E3C00FBE4C0E0C0037B027A0079E17D057C1DC8
:103E4C00780D12081D158115817F027B027A00798D
:103E5C00E11295A9023B6A7B027A0079E17D057C2F
:103E6C001D782012081D74069000E1F07F017B0282
:103E7C007A0079E11295A9900118E0B4010E7F0245
:103E8C007B057A1D79311295A90240447F027B058E
:103E9C007A1C79DA1295A9023B6A7B027A0079E1E5
:103EAC007D057C1D784212081D74069000E1F07FA0
:103EBC00017B027A0079E11295A990011EE0FEA324
:103ECC00E0FFE4FCFD121491C004C005C006C0075D
:103EDC0074CDFC14FDFE743DFF12112C79271200D9
:103EEC00F490011DE0FF129CBAE4FCFD121491C089
:103EFC0004C005C006C00779271200E8121288C05A
:103F0C0004C005C006C00790011DE0FBE4C0E0C082
:103F1C00037B027A0079E17D057C1D785312081D24
:103F2C0074FA2581F5817F027B027A0079E1129582
:103F3C00A9023B6A7B027A0079E17D057C1D7866DB
:103F4C0012081D74069000E1F07F017B027A007963
:103F5C00E11295A990011EE0FEA3E0FFE4FCFD1226
:103F6C001491C004C005C006C00774CDFC14FDFE3E
:103F7C00743DFF12112C79271200F47F05129CBAA4
:103F8C00E4FCFD121491C004C005C006C0077927DB
:103F9C001200E8121288C004C005C006C0079001C8
:103FAC001EE0C0E0A3E0C0E07B027A0079E17D0571
:103FBC007C1D787712081D74FA2581F5817F027BB0
:103FCC00027A0079E11295A9023B6A7B027A0079A8
:103FDC00E17D057C1D788712081D74069000E1F0C8
:103FEC007F017B027A0079E11295A9900120E0B45F
:103FFC00010D7F027B057A1D79311295A980397FDD
:10400C00027B057A1C79DA1295A9023B6A7B027A4B
:10401C000079E17D057C1D789812081D74069000CE
:10402C00E1F07F017B027A0079E11295A97F027B96
:0B403C00057A1979331295A9023B6A3E
:07404700782BEFF21207F5E0
:10404E00129672EF792CF3792BE3B40B0040030236
:10405E0048C9FA232A9040677302408A02414602F9
:10406E0042020242A002434D024448024525024547
:0C407E00C002465002473902483E80C490
:10408A007F017B057A1D79A91295A990010EE0C0DE
:10409A00E0A3E0C0E07B027A0079E17D057C1C7830
:1040AA006312081D1581158174069000E1F07F02E4
:1040BA007B027A0079E11295A9792CE3B401209068
:1040CA00010EE0B40106A3E0B4F401D3401190015B
:1040DA000FE024FBFB90010EE034FFF0A3EBF07934
:0540EA002CE3B40227E5
:0740EF00900115E0B4011C73
:1040F600129B09E4FE7F0D129B62E4FE7F0D900188
:104106000EE0FCA3E0FD129A3F129B8A12965F22F4
:10411600792CE3B4030280030248C990010EE0B48F
:104126000905A3E0B4C40040030248C990010FE0AA
:104136002405FB90010EE03400F0A3EBF002404EA4
:104146007F017B057A1D79BA1295A9900109E0C015
:10415600E0A3E0C0E07B027A0079E17D057C1C7873
:104166006312081D1581158174069000E1F07F0227
:104176007B027A0079E11295A9792CE3B4012090AB
:104186000109E0B40106A3E0B4F401D340119001A3
:104196000AE024FBFB900109E034FFF0A3EBF07981
:0541A6002CE3B4022728
:0741AB00900115E0B4011CB6
:1041B200129B09E4FE7F06129B62E4FE7F069001D9
:1041C20009E0FCA3E0FD129A3F129B8A12965F223D
:1041D200792CE3B4030280030248C9900109E0B4D8
:1041E2000905A3E0B4C40040030248C990010AE0F3
:1041F2002405FB900109E03400F0A3EBF002404EED
:104202007F017B057A1D79CB1295A990011AE0FBFB
:10421200E4C0E0C0037B027A0079E17D057C1C7872
:104222009512081D1581158174069000E1F07F0238
:104232007B027A0079E11295A9792CE3B4011090FE
:10424200011AE0B41E01D3400690011AE014F0797D
:054252002CE3B402267C
:07425700900115E0B4011B0A
:10425E00129B09E4FE7F0B129B62E4FE7F0B900122
:10426E001AE0FD7C00129A3F129B8A12965F227909
:10427E002CE3B4030280030248C990011AE0FB7AD2
:10428E0000B4F00040030248C990011AE004F002A5
:10429E00404E7B027A0079E17D057C1D78DC1208A8
:1042AE001D7F017B027A0079E11295A990010DE044
:1042BE00FBE4C0E0C0037B027A0079E17D057C1C43
:1042CE00789512081D1581158174069000E1F07F16
:1042DE00027B027A0079E11295A9792CE3B40110E0
:1042EE0090010DE0B41E01D3400690010DE014F0D4
:0642FE00792CE3B4022656
:07430400900115E0B4011B5C
:10430B00129B09E4FE7F0C129B62E4FE7F0C900172
:10431B000DE0FD7C00129A3F129B8A12965F227968
:10432B002CE3B4030280030248C990010DE0FB7A31
:10433B0000B4F00040030248C990010DE004F00204
:10434B00404E7F017B057A1D79ED1295A9900113E3
:10435B00E0FAA3E0FBBA0704B46C01D3503CE4FCD5
:10436B00FDAE02AF03121491C004C005C006C00716
:10437B007C6F7D127E837F3A12112CC004C005C066
:10438B0006C0077B027A0079E17D057C1D78FE1261
:10439B00081D74FC2581F581800F7B027A0079E181
:1043AB007D057C1C78DA12081D74069000E1F07F05
:1043BB00027B027A0079E11295A9792CE3B40120F2
:1043CB00900113E0B40606A3E0B44001D340119072
:1043DB000114E024F6FB900113E034FFF0A3EBF0A3
:0643EB00792CE3B4022767
:0743F100900115E0B4011C6E
:1043F800129B09E4FE7F05129B62E4FE7F05900193
:1044080013E0FCA3E0FD129A3F129B8A12965F22EA
:10441800792CE3B4030280030248C9900113E0B485
:104428000705A3E0B4760040030248C9900114E0F0
:10443800240AFB900113E03400F0A3EBF002404E95
:104448007F017B057A1E790F1295A9900110E0FE75
:10445800A3E0FFE4FCFD121491C004C005C006C02F
:10446800077C6F7D127E837F3A12112CC004C00531
:10447800C006C0077B027A0079E17D057C1D78FEC5
:1044880012081D74FC2581F58174069000E1F07F07
:10449800027B027A0079E11295A9792CE3B4012014
:1044A800900110E0B40106A3E0B4F401D3401190E8
:1044B8000111E024F6FB900110E034FFF0A3EBF0CB
:0644C800792CE3B4022789
:0744CE00900115E0B4011C90
:1044D500129B09E4FE7F08129B62E4FE7F089001AF
:1044E50010E0FCA3E0FD129A3F129B8A12965F2210
:1044F500792CE3B4030280030248C9900110E0B4AB
:104505000405A3E0B4B00040030248C9900111E0DE
:10451500240AFB900110E03400F0A3EBF002404EBA
:104525007F017B057A1E79201295A9900117E0FB82
:10453500E4C0E0C0037B027A0079E17D057C1E784A
:104545003112081D1581158174069000E1F07F0276
:104555007B027A0079E11295A9792CE3B4011090D8
:104565000117E0B40501D34006900117E014F07976
:054575002CE3B4022656
:07457A00900115E0B4011BE4
:10458100129B09E4FE7F09129B62E4FE7F09900100
:1045910017E0FD7C00129A3F129B8A12965F2279E6
:1045A1002CE3B4030280030248C9900117E0B41957
:1045B1000040030248C9900117E004F002404E7F19
:1045C100017B057A1E79431295A9900118E0B40187
:1045D100117B027A0079E17D057C1E785412081D59
:1045E100800F7B027A0079E17D057C1E78651208D7
:1045F1001D74069000E1F07F027B027A0079E112DE
:0D46010095A9792CE364016004E3B4031172
:10460E00900118E0B40104E4F080067401900118E2
:0C461E00F0792CE3B4020280030248C9CA
:07462A00900115E0B4011B33
:10463100129B09E4FE7F0F129B62E4FE7F0F900143
:1046410018E0FD7C00129A3F129B8A12965F227F2E
:10465100017B057A1E79761295A990011EE0FEA3D1
:10466100E0FFE4FCFD121491C004C005C006C007C0
:1046710074CDFC14FDFE743DFF12112C9000B2129A
:1046810000D090011DE0FF129CBAE4FCFD121491D0
:10469100C004C005C006C0079000B2121285C00454
:1046A100C005C006C00790011DE0FBE4C0E0C003E7
:1046B1007B027A0079E17D057C1D785312081D7417
:1046C100FA2581F58174069000E1F07F027B027A80
:1046D1000079E11295A9792CE3B4011090011DE054
:1046E100B40001D3400690011DE014F0792CE3B42D
:0246F10002269F
:0746F300900115E0B4011B6A
:1046FA00129B09E4FE7F04129B62E4FE7F04900190
:10470A001DE0FD7C00129A3F129B8A12965F227965
:10471A002CE3B4030280030248C990011DE0B404EB
:10472A000040030248C990011DE004F002404E7F98
:10473A00017B057A1E79871295A990011EE0FEA3D6
:10474A00E0FFE4FCFD121491C004C005C006C007D6
:10475A0074CDFC14FDFE743DFF12112C9000B212B0
:10476A0000D07F05129CBAE4FCFD121491C004C06B
:10477A0005C006C0079000B2121285C004C005C069
:10478A0006C00790011EE0C0E0A3E0C0E07B027A09
:10479A000079E17D057C1D787712081D74FA258160
:1047AA00F58174069000E1F07F027B027A0079E1DC
:1047BA001295A9792CE3B4011E90011EE0B40706F4
:1047CA00A3E0B4D001D3400F90011FE014F0F4909D
:0D47DA00011E7003E014F0792CE3B40227F7
:0747E700900115E0B4011C74
:1047EE00129B09E4FE7F07129B62E4FE7F07900195
:1047FE001EE0FCA3E0FD129A3F129B8A12965F22E6
:10480E00792CE3B4030280030248C990011EE0B480
:10481E000B05A3E0B4B80040030248C990011FE0A5
:10482E0004F090011E60030248C9E004F002404EFD
:10483E007F017B057A1E79981295A9900120E0B42C
:10484E0001117B027A0079E17D057C1E78541208F5
:10485E001D800F7B027A0079E17D057C1E78651242
:10486E00081D74069000E1F07F027B027A0079E168
:0E487E001295A9792CE364016004E3B40311E0
:10488C00900120E0B40104E4F08006740190012052
:07489C00F0792CE3B40226C1
:0748A300900115E0B4011BB8
:1048AA00129B09E4FE7F0A129B62E4FE7F0A9001D2
:1048BA0020E0FD7C00129A3F129B8A12965F220228
:0248CA00404E5E
:1048CC002053746172742043686172676572202092
:1048DC00002053746172742054726967676C652090
:1048EC0020002020202020202020202020202025D7
:1048FC0032642000205374617274204469736368BD
:05490C00617267650007
:10491100782DEEF208EFF2782FEDF28D0712504B61
:10492100EE9000C5F0A3EFF0900132E0FBE49000BF
:10493100BFF0A3EBF0E4FDFC9000B7F090011EE0A6
:10494100FEA3E0FF1214919000B91200D0E4FCFD27
:104951009000DFE0FEA3E0FF121491C004C005C087
:1049610006C0077C6F7D127E837F3A12112CC00432
:10497100C005C006C0079000D5E0FF7E00E433E427
:10498100500114FCFD12145412112CC004C005C0B6
:1049910006C0079000B9121129121495EE9000C1BA
:1049A100F0A3EFF0792FE324FD7003024C6514703E
:0F49B10003024C6524FE600714600414600122A9
:1049C000900120E0B40103120003792FE3FF12509D
:1049D0004BEE9000BDF0A3EFF070189000BDE070BA
:1049E000129000C5E0FAA3E0FB9000BDEAF0A3EB53
:1049F000F080109000BDE0FAA3E0FB9000C5EAF063
:104A0000A3EBF0E4FCFD792DE3FE09E3FF12149122
:104A1000C004C005C006C0077C0A7DD77EA37F3CCA
:104A200012112C121495EE9000C3F0A3EFF0792F21
:0E4A3000E364066009E3B408028003024AE270
:104A3E009000B8E0F5F0900130E065F07003024AA6
:014A4E00E285
:104A4F00E09000B8F0792FE3B406117B027A007979
:104A5F00E17D057C4878CC12081D800F7B027A001F
:104A6F0079E17D057C4878DD12081D74069000E120
:104A7F00F07F017B027A0079E11295A9E5FEFF7EB6
:104A8F0000E4FC7D6412013DE4FC7DFF120151C086
:104A9F0006C0077B027A0079E17D057C4878EE122B
:104AAF00081D15811581792D900035E3F009A3E3D9
:104ABF00F07B027A0079E19000BDE0FCA3E0FD12EB
:104ACF0050AF74259000F0F07F027B027A0079E1FD
:104ADF001295A9E5FE9000B6F09000BDE0FAA3E0B4
:104AEF00FBEAFEEBFF9000C4E0FC792EE3C39CFDD4
:104AFF009000C3E0FB19E39BFCF5F0EAB5F004EF7F
:104B0F00B50500500CE5FEFB7A00B4F3005002052A
:104B1F00FE9000BDE0FAA3E0FB9000C4E0FC792E0C
:104B2F00E32CFF9000C3E0FD19E33DFEF5F0EAB57D
:104B3F00F005EBB50701D3400AE5FEB40001D34001
:104B4F000215FE9000BDE0FEA3E0FF9000C4E0FA66
:104B5F00792EE3C39AFB9000C3E0FC19E39CFAF5AE
:104B6F00F0EEB5F004EFB50300401EA3E0F809E343
:104B7F0028FB9000C3E0F819E338FAF5F0EEB5F032
:104B8F0005EFB50301D3500122E5FEB40101D34077
:104B9F000AE5FEFB7A00B4F20040099000BDE0FE8A
:0E4BAF00A3E0FF229000B6E0B5FE01D3401552
:104BBD009000B7E004F0B40A01D340099000BDE0C5
:0F4BCD00FEA3E0FF229000DEE0B40101D34049D7
:104BDC00125093E4FCFD121491C004C005C006C031
:104BEC0007E4FCFD9000C1E0FEA3E0FF121491C0AD
:104BFC0004C005C006C0079000B9120089E4FEFC91
:104C0C00FD743FFF12112C120FCC121522BF01099B
:104C1C009000BDE0FEA3E0FF22792FE3B4070280F1
:044C2C00030249C076
:104C30003080032081099000BDE0FEA3E0FF2290B8
:104C400000BFE0FCA3E0FD900132E0FB7A008AF0B7
:104C5000BC0009F5F0ED6B70030249C09000BDE0A7
:054C6000FEA3E0FF22AD
:104C6500900120E0B40103120003792FE3FF1250F5
:104C75004BEE9000BDF0A3EFF070189000BDE07012
:104C8500129000C5E0FAA3E0FB9000BDEAF0A3EBAB
:104C9500F080109000BDE0FAA3E0FB9000C5EAF0BB
:104CA500A3EBF0E4FCFD792DE3FE09E3FF1214917B
:104CB500C004C005C006C0077C0A7DD77EA37F3C23
:104CC50012112C121495EE9000C3F0A3EFF0792F7A
:094CD500E3B403028003024D6800
:0E4CDE009000B8E0F5F0900130E065F0607CE9
:104CEC00E09000B8F07B027A0079E17D057C497890
:104CFC000012081D74069000E1F07F017B027A001F
:104D0C0079E11295A9E5FDFF7E00E4FC7D641201BA
:104D1C003DE4FC7DFF120151C006C0077B027A0006
:104D2C0079E17D057C4878EE12081D158115817995
:104D3C002D900035E3F009A3E3F07B027A0079E1D2
:104D4C009000BDE0FCA3E0FD1250AF74259000F084
:104D5C00F07F027B027A0079E11295A9E5FD9000C3
:104D6C00B6F09000BDE0FAA3E0FB9000C4E0FC7943
:104D7C002EE3C39CFD9000C3E0F819E398FCF5F01A
:104D8C00EAB5F004EBB50500500CE5FDFB7A00B478
:104D9C00F300500205FD9000BDE0FAA3E0FB90008B
:104DAC00C4E0FC792EE32CFF9000C3E0FD19E33D39
:104DBC00FEF5F0EAB5F005EBB50701D3400AE5FDC9
:104DCC00B40001D3400215FD9000BDE0FCA3E0FD52
:104DDC009000C4E0FA792EE3C39AFB9000C3E0F88C
:104DEC0019E398FAF5F0ECB5F004EDB503004022A8
:104DFC00ECFEEDFFA3E0F809E328FB9000C3E0FD17
:104E0C0019E33DFAF5F0ECB5F005EFB50301D3501D
:104E1C000122E5FDB40101D3400AE5FDFB7A00B4A3
:104E2C00F20040099000BDE0FEA3E0FF229000B626
:074E3C00E0B5FD01D34015B4
:104E43009000B7E004F0B40A01D340099000BDE03C
:104E5300FEA3E0FF22792FE3B404028003024C6532
:104E63003080032081099000BDE0FEA3E0FF229083
:104E730000BFE0FCA3E0FD900132E0FB7A008AF082
:104E8300BC0009F5F0ED6B7003024C659000BDE0CA
:054E9300FEA3E0FF2278
:104E98007830EEF208EFF2900132E0FBE49000CDBA
:104EA800F0A3EBF0125093EE9000C7F0A3EFF0E4FC
:104EB800FCFD90011EE0FEA3E0FF1214919000C9D2
:034EC8001200D005
:104ECB00900120E0B40103120003125093EE900006
:104EDB00D1F0A3EFF070189000D1E070129000C7E2
:104EEB00E0FAA3E0FB9000D1EAF0A3EBF080109086
:104EFB0000D1E0FAA3E0FB9000C7EAF0A3EBF0903F
:104F0B0000DEE064026009E064036004E0B4041EA8
:104F1B009000C91200897C0A7DD77EA37F3B1211BA
:104F2B002C121495EE9000CFF0A3EFF0801C9000A4
:104F3B00C91200897C0A7DD77EA37F3C12112C12EB
:104F4B001495EE9000CFF0A3EFF09000D1E0FCA30E
:104F5B00E0FD9000D0E0FA7931E3C39AFB9000CFEB
:104F6B00E0F819E398FAF5F0ECB5F004EDB50300B1
:104F7B00500CE5FEFB7A00B4F300500205FE9000E6
:104F8B00D1E0FEA3E0FF9000D0E0FA7931E32AFDF7
:104F9B009000CFE0FB19E33BFCF5F0EEB5F005EF2D
:104FAB00B50501D3400AE5FEB40001D3400215FE5E
:104FBB009000D1E0FEA3E0FF9000D0E0FA7931E35E
:104FCB00C39AFB9000CFE0FC19E39CFAF5F0EEB529
:104FDB00F004EFB50300401EA3E0F809E328FB90B3
:104FEB0000CFE0F819E338FAF5F0EEB5F005EFB5C0
:104FFB000301D3500122E5FE64016006E5FE64F275
:10500B0070099000D1E0FEA3E0FF223080032081E5
:10501B00099000D1E0FEA3E0FF229000CDE0FCA3BD
:10502B00E0FD900132E0FB7A008AF0BC0009F5F05C
:10503B00ED6B7003024ECB9000D1E0FEA3E0FF229C
:08504B007832EFF2E47933F34F
:105053007932E324FD601214601E24FE600514609F
:035063000E801E9E
:105066007F06129CBA227F07129CBA2220970F7FD6
:1050760006129CBA222096067F07129CBA22793322
:0D508600E304F37933E3B464C4E4FEFF22D5
:04509300E47934F395
:105097002097067F05129CBA227934E304F379340A
:0850A700E3B464ECE4FEFF2217
:1050AF007837EBF208EAF208E9F2783AECF208ED19
:1050BF00F2E4FCFD793AE3FE09E3FF121491C00418
:1050CF00C005C006C007E4FCFD74C8FE7442FF12A1
:1050DF00112CC004C005C006C007E4FCFD7835E202
:1050EF00FE08E2FF121491121288121495EF783C09
:1050FF00F27937783DE3F20908E3F20908E3F27831
:0F510F003DE2FB08E2FA08E2F9E41200427F01F8
:10511E00793FE304F3197003E304F3793DE3FD09EA
:10512E00E3FC09E3F874011200260FBF09E2793F90
:10513E00E304F3197003E304F3793DE3FD09E3FCA3
:0C514E0009E3F87402120026E47940F333
:10515A007940E3FF7E00E4FC7D0A12013D8EF0797E
:10516A003CE3FBB2F77480B5F005EBB50701D34019
:01517A0056DE
:10517B007937E3FD09E3FC09E3F8740312002679A0
:10518B0039E304F3197003E304F37940E3B4080043
:10519B0050107937E3FD09E3FC09E3F8E41200262C
:1051AB00800F7937E3FD09E3FC09E3F87403120080
:1051BB00267940E3B4090F7937E3FD09E3FC09E3F2
:1051CB00F874201200267940E304F37940E3B40A23
:0751DB0002800302515A2279
:1051E20075FA0075EA0075DA0075FB0075EB00755B
:1051F200DB0075FC0075EC0075DC0075FD0075EDDB
:105202000075DD0075FE0075EE0075DE00C2DED2AF
:0A52120093D294D295D296D297223F
:10521C00C0E0C083C082C0D0C002C003758C87754B
:0B522C008AFF900131E0B4640050469E
:10523700E004F09000D8E0FAA3E0BA0004B400015B
:10524700D3400CE014F0F49000D87003E014F09011
:065257000131E0B4325FFA
:10525D00900130E070057401F08005E4900130F0AC
:10526D0090012FE004F0B40401D34043E4F0803FFB
:10527D00E4900131F0A3E004F0A3E0FAA3E0BA005A
:10528D0004B40001D3400CE014F0F490013370032A
:10529D00E014F0900137E0FAA3E0BA0004B4000185
:1052AD00D3400CE014F0F49001377003E014F0904B
:0952BD000132E0B43B01D34010C2
:1052C600E4F0900136E004F09001357003E004F05C
:0D52D600D003D002D0D0D082D083D0E032FF
:1052E300204368617267657220526573657420207C
:1052F300002066726F6D205761746368646F672165
:10530300200020202057454C434F4D4520544F202B
:1053130020200020534D41525420434841524745D9
:1053230052202000436F70797269676874202843A4
:1053330029204279007777772E686F6262792D7220
:10534300632E636F6D0020496E697469616C204D33
:10535300656D6F7279200020506C6561736520570D
:105363006169742E2E2E200020202A2A20455252B5
:105373004F52202A2A2020200020204D656D6F7275
:1053830079204661696C202020004C6F6164696E4E
:10539300672042617474657279200046726F6D20D4
:1053A3004C6F636174696F6E2025326400204C6F0B
:1053B3006164696E672044656661756C7400534D62
:1053C30041525420434841524745522042592050AC
:1053D300484F454E49582400436F70797269676896
:1053E300742028432920323030362E204279205031
:1053F300484F454E49582400687474703A2F2F77EC
:1054030077772E686F6262792D72632E636F6D24D6
:10541300004649524D574152452056455253494F34
:105423004E20312E313861240044495343484152C0
:1054330047453A202400253364204D494E3A202421
:105443000056424154543D25352E3266563A2024A7
:105453000049424154543D25352E3266413A2024B9
:105463000050574D3D2532642020240043484152CB
:1054730047453A20202020240054494D45523D25DC
:105483003464204D494E3A202400204261747465EF
:1054930072792046756C6C79202000204368617214
:1054A30067652044657465637421200043686172F5
:1054B3006765722066756E6374696F6E0069732029
:1054C30064697361626C65642E2020202000446946
:1054D3007363682E2066756E6374696F6E20002097
:1054E3002020202025326443202534646D41680048
:1054F30020204E6F20426174746572792020202031
:1055030000202025352E3266562025352E3266564C
:10551300730053544F502044495343484152474525
:10552300523F0020444953434841524745202020DD
:105533002020200020202057616974202533642017
:105543007365632E004449534348415247453A200B
:10555300424154544552593D2400202020203A20F2
:10556300240043415041434954593D2534646D411E
:10557300683A20240043454C4C3D2532643A2024AC
:10558300004944495343483D25352E3266412400A2
:105593002053746172742044697363686172676530
:1055A3000020202020202020202020202020202018
:1055B3002000202020202020202020252B34646D53
:1055C30041680025352E3266562025332E3166413B
:1055D30020253364730025352E3266562025332E5D
:1055E300316641202533646D0025352E32665673AE
:1055F300202050574D20253264200053544F502013
:10560300434841524745523F202020002043484110
:1056130052474520202020202020202020004348DE
:10562300415247453A20424154544552593D240082
:10563300494348415247453D25352E3266413A207C
:105643002400494D494E5F54483D2532646D413A2B
:1056530020240054494D45523D2535643A20240009
:1056630020537461727420436861726765722020ED
:105673000025352E326656202532646D41202533B0
:1056830064730025352E326656202532646D412021
:105693002533646D002054524947474C4520252B40
:1056A30034646D4168002046554C4C5920434841B1
:1056B3005247452020200020444953434841524744
:1056C3004520444F4E452000205553455220544514
:1056D300524D494E415445440020424154542E20DA
:0A56E3004F5645522D564F4C54000F
:1056ED00204241545420444953434F4E4E45435458
:1056FD0000204C4F5720535550504C5920564F4C6D
:10570D0054002044495343482E2020252B34646DEA
:10571D004168002044495343482E54494D452025A6
:10572D0033646D00204348415247452020252B34DA
:10573D00646D416800204348472E54494D45202053
:10574D00202533646D00204D4554484F443A204385
:10575D00432D4356202000204D4554484F443A20B8
:10576D004E45472D64562000204D4554484F443A30
:10577D0020494E464C45582000204D4554484F4435
:10578D003A2054494D4552202000204D4554484F54
:10579D00443A205A45524F2D6456002025352E325D
:1057AD006656702025352E326656652000205355DD
:1057BD0050504C59202025352E326656732000202E
:1057CD0020204E6F2020202020596573202020009E
:1057DD007580FF7590FF75A0FF75B0FFE4FE7FFA31
:1057ED001296471294761207F5E4FF12956A7589A1
:1057FD0021758C87758AFF75985253877F758DFB40
:10580D00D28CD28E75A8921207EB1251E2129A36F3
:09581D0030C23A900120E0603431
:1058260012026C7F017B057A5279E31295A97F02F9
:105836007B057A5279F41295A9C2B430801430816E
:015846001150
:1058470020B40312960B7E017FF4129647B2B48000
:10585700E9D2B4308007208104D2008002C2007FE1
:10586700017B057A5379051295A97F027B057A5347
:1058770079161295A97E077FD01296477F017B057F
:105887007A5379271295A97F027B057A53793812C3
:1058970095A97E037FE8129647740190010CF0905A
:1058A7000116F090011CF07404A3F0900113740723
:1058B700F0A37476F09001097404F0A374B0F0902B
:1058C700011E7408F0A37484F09001107403F0A310
:1058D70074E8F0740F900117F07401900120F074D0
:1058E7003C90011AF090010DF0A37404F0A374B07A
:1058F700F0E4FFFE900112F0900118F0A3F0900180
:105907001BF0129A78BE01028003025A10BF0002F0
:055917008003025A109C
:10591C007401900115F0E4FE7F01129A78EF90016A
:10592C000CF0E4FE7F02129A78EF900146F0540FCF
:10593C00900116F0900146E05480B40800E4400158
:10594C0004900119F0900146E05440B40700E44083
:10595C00010490011BF0E4FE7F03129A78EF900192
:10596C001CF0E4FE7F04129A78EF90011DF0E4FE27
:10597C007F05129A78EE900113F0A3EFF0E4FE7F0E
:10598C0006129A78EE900109F0A3EFF0E4FE7F077F
:10599C00129A78EE90011EF0A3EFF0E4FE7F08124D
:1059AC009A78EE900110F0A3EFF0E4FE7F09129AC2
:1059BC0078EF900117F0E4FE7F0A129A78EF9001CD
:1059CC0020F0E4FE7F0B129A78EF90011AF0E4FEBF
:1059DC007F0C129A78EF90010DF0E4FE7F0D129A75
:1059EC0078EE90010EF0A3EFF0E4FE7F0E129A78A1
:1059FC00EF900112F0E4FE7F0F129A78EF900118ED
:045A0C00F0025B97B2
:105A10007F017B057A5379491295A97F027B057A2C
:105A200053795A1295A9129B09E4FE7F0A129647F0
:105A3000E4FEFF129B62E4FDFEFF7C01129A3F121E
:105A40009B8AE4FEFF129A78BE01028003025B6823
:085A5000BF00028003025B6845
:105A58007401900115F0129B09E4FE7F0A12964723
:105A6800E4FE7F0190010CE0FD7C00129A3F90015A
:105A780016E0900146F0900119E0B4010790014644
:105A8800E04480F090011BE0B40107900146E04437
:105A980040F0E4FE7F02900146E0FD7C00129A3F50
:105AA800E4FE7F0390011CE0FD7C00129A3FE4FEB7
:105AB8007F0490011DE0FD7C00129A3FE4FE7F0503
:105AC800900113E0FCA3E0FD129A3FE4FE7F0690EC
:105AD8000109E0FCA3E0FD129A3FE4FE7F07900174
:105AE8001EE0FCA3E0FD129A3FE4FE7F089001103F
:105AF800E0FCA3E0FD129A3FE4FE7F09900117E065
:105B0800FD7C00129A3FE4FE7F0A900120E0FD7CB4
:105B180000129A3FE4FE7F0B90011AE0FD7C001210
:105B28009A3FE4FE7F0C90010DE0FD7C00129A3F45
:105B3800E4FE7F0D90010EE0FCA3E0FD129A3FE425
:105B4800FE7F0E900112E0FD7C00129A3FE4FE7F7A
:105B58000F900118E0FD7C00129A3F129B8A802F5B
:105B6800E4900115F07F017B057A53796B1295A9B2
:105B78007F027B057A53797C1295A912965FE4FE21
:105B88007FC812964712965F7E027FBC1296471214
:0B5B980091D330800C20810930000602
:105BA30012965F123B29900115E0B40102800302B3
:025BB3005DCBC8
:105BB500900112E0B401005003025D23E0B40A0134
:065BC500D34003025D2342
:105BCB00E0FB24FFFFE434FFFEE4FC7D0A12013D01
:105BDB00EF2410FFE43E9001A6F0A3EFF0EB2400BE
:105BEB00FBE43455FAC002C0039001A6E0FEA3E02B
:105BFB00FF129A78D005D0F0EEB5F0028003025C6C
:0A5C0B00DBEFB505028003025CDB4D
:105C15007F017B057A53798D1295A9900112E0FBDE
:105C2500E4C0E0C0037B027A0079E17D057C53780E
:105C35009E12081D158115817F027B027A0079E18C
:105C45001295A99001A7E02401FF9001A6E0340078
:105C5500FE129A78EF9000DEF09001A7E02402FF93
:105C65009001A6E03400FE129A78EE9000D3F0A3DE
:105C7500EFF09001A7E02403FF9001A6E03400FEB9
:105C8500129A78EF9000D5F09001A7E02404FF90D8
:105C950001A6E03400FE129A78EE9000DAF0A3EF48
:105CA500F09001A7E02405FF9001A6E03400FE1264
:105CB5009A78EE9000DCF0A3EFF09001A7E02406BF
:105CC500FF9001A6E03400FE129A78EE9000DFF016
:065CD500A3EFF0025DCB1D
:105CDB007F017B057A5379B01295A97F027B057AF8
:105CEB0053795A1295A9E49000DEF09000D3740317
:105CFB00F0A374E8F07408A3F09000DA7403F0A337
:105D0B0074E8F0A37401F0A374F4F09000DF740551
:085D1B00F0A37478F0025DCBE7
:105D23007F017B057A5379B01295A97F027B057AAF
:105D330053795A1295A9E4FE7F10129A78BE5559E9
:035D4300BF015647
:105D4600E4FE7F11129A78EF9000DEF0E4FE7F12F7
:105D5600129A78EE9000D3F0A3EFF0E4FE7F1312D0
:105D66009A78EF9000D5F0E4FE7F14129A78EE90C0
:105D760000DAF0A3EFF0E4FE7F15129A78EE9000B9
:105D8600DCF0A3EFF0E4FE7F16129A78EE9000DFC7
:065D9600F0A3EFF0802FE6
:105D9C00E49000DEF09000D37403F0A374E8F07488
:105DAC0008A3F09000DA7403F0A374E8F0A3740174
:105DBC00F0A374F4F09000DF7405F0A37478F09005
:105DCC0000DEE0B40101D340067402900116F0E449
:105DDC00900131F0900135F0A3F0900132F0D2A98E
:105DEC001294439000D6E4F0A3F00490010BF0C29F
:105DFC000190014FF0E4FDFC900152F0900109E09C
:105E0C00FEA3E0FF121491C004C005C006C0077CBD
:105E1C006F7D127E837F3A12112C9001391200D0C3
:105E2C00E4FCFD90010EE0FEA3E0FF121491C0040F
:105E3C00C005C006C0077C6F7D127E837F3A1211AD
:105E4C002C90013D1200D0E4FCFD90011EE0FEA35D
:105E5C00E0FF121491C004C005C006C00774CDFC4D
:105E6C0014FDFE743DFF12112C9001411200D075EF
:105E7C00FD7F75ED7F75DD42D2DE7E037FE81296E5
:105E8C00471251E212965F1207F5900120E0B4011F
:0E5E9C0003120262900118E0B40001D34065C9
:105EAA007F0D1296DB7F0A1296DB7F0A1296DB7B46
:105EBA00057A5379C11296EA7F0D1296DB7F0A1290
:105ECA0096DB7B057A5379DB1296EA7F0D1296DB15
:105EDA007F0A1296DB7F0A1296DB7B057A5379FBDF
:105EEA001296EA7F0D1296DB7F0A1296DB7F0A1260
:105EFA0096DB7B057A5479141296EA7F0D1296DBAB
:055F0A007F0A1296DB86
:105F0F0090014EE0FB7A008AF0900135E0FCA3E0AF
:105F1F00FDBC00088BF06B7003026165900118E007
:095F2F00B40001D35003026165C6
:0F5F3800ED90014EF0A3E0B4040280030260502C
:105F47007F0D1296DB7F0A1296DB7B057A54792C3C
:105F57001296EA900135E0C0E0A3E0C0E07B027A48
:105F67000079E17D057C54783912081D158115816A
:105F77007B027A0079E11296EAE4FCFD90015AE08F
:105F8700FEA3E0FF121491C004C005C006C007902D
:105F97000141121285C004C005C006C0077B027A02
:105FA7000079E17D057C54784412081D74FC258135
:105FB700F5817B027A0079E11296EAE4FCFD900113
:105FC70054E0FEA3E0FF121491C004C005C006C050
:105FD70007900139121285C004C005C006C0077CAE
:105FE7006F7D127E837F3A12112CC004C005C00654
:105FF700C0077B027A0079E17D057C54785412084A
:106007001D74FC2581F5817B027A0079E11296EAFD
:10601700E5FDFF7E00E4FC7D6412013DE4FC7DFFAD
:10602700120151C006C0077B027A0079E17D057C29
:1060370054786412081D1581158174259000E7F0C6
:106047007B027A0079E11296EA90014FE0B40702E9
:056057008003026165F9
:10605C007F0D1296DB7F0A1296DB7B057A54796FE3
:10606C001296EA900137E0C0E0A3E0C0E07B027A30
:10607C000079E17D057C54787C12081D1581158111
:10608C007B027A0079E11296EAE4FCFD90015AE079
:10609C00FEA3E0FF121491C004C005C006C0079017
:1060AC000141121285C004C005C006C0077B027AEC
:1060BC000079E17D057C54784412081D74FC25811F
:1060CC00F5817B027A0079E11296EAE4FCFD9001FD
:1060DC0054E0FEA3E0FF121491C004C005C006C03A
:1060EC0007900139121285C004C005C006C0077C98
:1060FC006F7D127E837F3A12112CC004C005C0063E
:10610C00C0077B027A0079E17D057C547854120833
:10611C001D74FC2581F5817B027A0079E11296EAE7
:10612C00E5FEFF7E00E4FC7D6412013DE4FC7DFF96
:10613C00120151C006C0077B027A0079E17D057C13
:10614C0054786412081D1581158174259000E7F0B0
:10615C007B027A0079E11296EA900120E0B4010307
:10616C00120003129672EF90014CF090014FE0B4C4
:10617C000503026F855014E0146028147003026547
:10618C00AF24FE700302692F0291D0E024F9700352
:10619C00027A9F24FE7003028B47147003028F1146
:0361AC00025F0F80
:1061AF00D2B2D2B3D2B490014CE0B4010280030258
:0861BF0062AC2001030262AC96
:0B61C700900116E06403700302628484
:1061D2009000DEE06009E0B40102800302625CE448
:1061E200FCFD90015AE0FEA3E0FF121491C004C02E
:1061F20005C006C007900141121285C004C005C047
:1062020006C0079000D5E0FB7A00E433E4500114A5
:10621200FCFDAE02AF03121454121288C004C00572
:10622200C006C0077CCD7DCC7EAC7F3F121522BF5D
:02623200012841
:10623400C2B41296347F017B057A54798D1295A9E4
:106244007F027B057A54799E1295A912965F7E0788
:086254007FD0129647025F0F94
:10625C00740190010BF0740590014FF0129443906F
:10626C00011AE0FBE4900133F0A3EBF0A3E4F0A3FC
:08627C00F0900132F0025F0F07
:10628400C2B41296347F017B057A5479AF1295A972
:106294007F027B057A5479C01295A912965F7E0716
:0F62A4007FD0129647025F0F90014CE0B40209C1
:1062B3001202691239D312000690014CE0B4035361
:0362C30030015057
:0862C600900116E06402602261
:1062CE00740290014FF012944390011AE0FBE49097
:1062DE000133F0A3EBF0A3E4F0A3F0900132F0024F
:0262EE0091D04D
:1062F0001296347F017B057A5479D11295A97F02D9
:106300007B057A5479C01295A912965F7E077FD0DB
:10631000129647025F0F7F05129CBAEE90015AF069
:0F632000A3EFF090010CE0B40102800302648D42
:10632F009000DEE0FAB403030263F5500CEA601A42
:10633F0014601714606202648DEA24FC7003026318
:0A634F00F514700302644202648D2D
:10635900E4FCFD90015AE0FEA3E0FF121491C00491
:10636900C005C006C007900141121285C004C005CE
:10637900C006C0077CF57DBE7E207F4012112CC06F
:1063890004C005C006C00774ABFC14FDFE743EFFD3
:1063990012112C121495EF9000D5F002648DE4FCD3
:1063A900FD90015AE0FEA3E0FF121491C004C0055C
:1063B900C006C007900141121285C004C005C0067D
:1063C900C0077CB07DDE7E687F3F12112CC004C0FF
:1063D90005C006C00774ABFC14FDFE743EFF121124
:1063E9002C121495EF9000D5F002648DE4FCFD9019
:1063F900015AE0FEA3E0FF121491C004C005C006D3
:10640900C007900141121285C004C005C006C0072B
:106419007C737D717E557F3F12112CC004C005C06D
:1064290006C00774ABFC14FDFE743EFF12112C125A
:106439001495EF9000D5F0804BE4FCFD90015AE0F3
:10644900FEA3E0FF121491C004C005C006C0079066
:106459000141121285C004C005C006C0077C207D19
:10646900527EC07F3F12112CC004C005C006C00770
:1064790074ABFC14FDFE743EFF12112C121495EF3F
:106489009000D5F09000D3E0C0E0A3E0C0E0A3E025
:10649900FBE4C0E0C0037B027A0079E17D057C540E
:1064A90078E212081D74FC2581F5819000D5E07011
:1064B9000674419000E7F07B027A0079E19000DEF2
:1064C900E0FD1293FF7F017B027A0079E11295A921
:1064D90090011DE0FF129CBAEE9001A8F0A3EFF025
:1064E900E4FCFD90015AE0FEA3E0FF121491C00400
:1064F900C005C006C007900141121285C004C0053D
:10650900C006C0077466FEFCFD743FFF121522BF6A
:0A651900FF0280069000D5E0701923
:106523007B027A0079E17D057C5478F312081D74AF
:09653300069000E1F0C201806550
:10653C00E4FCFD9001A8E0FEA3E0FF121491C0045E
:10654C00C005C006C007900141121285C004C005E9
:10655C00C006C007E4FCFD90015AE0FEA3E0FF1268
:10656C001491C004C005C006C007900141121285E9
:10657C00C004C005C006C0077B027A0079E17D0526
:10658C007C55780412081D74F82581F581740290ED
:10659C0000E1F0D2017F027B027A0079E11295A929
:1065AC00025F0FD2B3D2B41251E27F05129CBAE44F
:1065BC00FCFD121491C004C005C006C00790014137
:1065CC00121285C004C005C006C0077466FEFCFD2F
:0965DC00743FFF121522BFFF4AB3
:1065E500C201E4900149F0740A90014FF0E4900172
:1065F50051F07404900150F012965F1251E212941A
:10660500437F05129CBAEE900129F0A3EFF09001AB
:106615001DE0FF129CBAEE90012DF0A3EFF0900162
:1066250033E4F0A37404F0025F0F90014CE0B4036F
:0F66350007900133E4F0A3F090014CE0B4025958
:106644007B057A557915129308EF64016003029172
:01665400D075
:106655007F05129CBAEE900129F0A3EFF01251E2EA
:1066650012965FE4900149F0740A90014FF0E490AE
:106675000151F07402900150F012944390011DE015
:10668500FF129CBAEE90012DF0A3EFF0900133E4D8
:10669500F0A37404F0025F0F7B027A0079E17D05B7
:1066A5007C55782612081D7B027A0079EC9000DE75
:1066B500E0FD1293FF74069000E1F07F017B027A02
:1066C5000079E11295A9900133E0C0E0A3E0C0E0B4
:1066D5007B027A0079E17D057C55783712081D1516
:1066E50081158174029000E1F0900130E0B4010A57
:0A66F50074079000E2F0C2B28002C8
:1066FF00D2B27F027B027A0079E11295A990013321
:0D670F00E06003026921A3E060030269213C
:0D671C00900118E0B40001D3500302680E94
:106729007F0D1296DB7F0A1296DB7B027A0079E1F4
:106739007D057C55784812081D7B027A0079E112A3
:1067490096EA7B027A0079E17D057C55785D12082D
:106759001D7B027A0079E19000DEE0FD1293FF7B58
:10676900027A0079E11296EA9000D3E0C0E0A3E052
:10677900C0E07B027A0079E17D057C5578651208D5
:106789001D158115817B027A0079E11296EA900044
:10679900D5E0FDE4C0E0C0057B027A0079E17D0522
:1067A9007C55787812081D158115817B027A00794C
:1067B900E11296EA9000DCE0FEA3E0FFE4FCFD12A2
:1067C9001491C004C005C006C0077C6F7D127E838A
:1067D9007F3A12112CC004C005C006C0077B027A9B
:1067E9000079E17D057C55788412081D74FC2581AA
:1067F900F5817B027A0079E11296EA7F0D1296DB28
:106809007F0A1296DBC2B275FD0175ED0175DD4295
:10681900D2DE90013D120089E4FCFD9000DCE0FE2F
:10682900A3E0FF12149112112C121495EE90015647
:10683900F0A3EFF09000D6E4F0A3F0C0E0C0E0745C
:1068490061C0E07445C0E09000DAE0FEA3E0FFE437
:10685900FCFD121491121288C004C005C006C007BD
:10686900E4FCFD74C8FE7442FF12112C121495EE5B
:106879009000D8F0A3EFF07B027A0079E17D057CE6
:1068890055789312081D74069000E1F07F017B0290
:106899007A0079E11295A97F027B057A5579A412CC
:1068A90095A97F0112956A900156E0FEA3E0FF7D4C
:1068B90003124911EE900154F0A3EFF07F027B051A
:1068C9007A5579A41295A9E4FF12956A7404900186
:0B68D9004FF0E4900152F090014BF0F2
:1068E400900154E0FCA3E0FD90014BE0FA2AFB2464
:1068F4006AF582E43401F583ECF0A3EDF090015ADB
:10690400E0FCA3E0FDEB247EF582E43401F583ECA6
:10691400F0A3EDF090014BE004F0B40AC39001350C
:10692400E4F0A3F0900132F0025F0FC2B290014C88
:10693400E064016004E0B403067405900152F09031
:0969440000D8E0705DA3E0705979
:10694D009000D7E004F09000D67003E004F0E4C0AE
:10695D00E0C0E07461C0E07445C0E0E4FCFD90016E
:10696D0054E0FEA3E0FF121491C004C005C006C0A0
:10697D000790013D121285121288C004C005C00691
:10698D00C007E4FCFD74C8FE7442FF12112C1214F2
:10699D0095EE9000D8F0A3EFF090014CE0B40279A1
:1069AD007B057A557915129308EF64016003029106
:0169BD00D009
:1069BE007F05129CBAEE900129F0A3EFF01251E27E
:1069CE0012965FE4900149F0740A90014FF0E49042
:1069DE000151F07402900150F09000D6E0FAA3E05D
:1069EE00FB900125EAF0A3EBF0900135E0FAA3E06D
:1069FE002401FBE43A900127F0A3EBF090011DE097
:106A0E00FF129CBAEE90012DF0A3EFF0900133E44B
:106A1E00F0A37404F0025F0F900132E0F5F09001E4
:096A2E004DE065F07003026BE815
:106A3700900152E0B40001D34003E014F090011D2F
:106A4700E0FF129CBAEE9001A8F0A3EFF07F0412CA
:106A5700504BEE90017AF0A3EFF09001B0120100D5
:096A670000000000E490014BF076
:106A700090014BE025E0246CF582E43401F583E0DD
:106A8000FCA3E0FD90014BE0FA2AFF246AF582E4C2
:106A90003401F583ECF0A3EDF09001B0120089EF22
:106AA000246AF582E43401F583E0FEA3E0FFE4FC10
:106AB000FD1201289001B01200D090014BE004F0CB
:106AC000B408AD75F0039001B01200C412000E902E
:106AD0000154EEF0A3EFF0A3E0FEA3E0FFE4FCFD21
:106AE000121491C004C005C006C0077C0A7DD77E81
:106AF000A37F3C12112C121495EE900166F0A3EFC7
:106B0000F0900154E0FCA3E0FDA3E0FAA3E0FB90C9
:106B10000167E0F8EBC398FB900166E0F8EA98FAA9
:106B2000F5F0ECB5F004EDB50300401EE0FAA3E08B
:106B3000FB900157E02BFB900156E03AFAF5F0ECA0
:0A6B4000B5F005EDB50301D34015D3
:106B4A00900156E0FEA3E0FF7D04124911EE900188
:106B5A0054F0A3EFF0125093EE90018EF0A3EFF0F1
:0F6B6A009001B012010000000000E490014BF018
:106B790090014BE025E02480F582E43401F583E0BF
:106B8900FCA3E0FD90014BE0FA2AFF247EF582E4A4
:106B99003401F583ECF0A3EDF09001B0120089EF18
:106BA900247EF582E43401F583E0FEA3E0FFE4FCF2
:106BB900FD1201289001B01200D090014BE004F0C1
:106BC900B408AD75F0039001B01200C412000E9024
:106BD900015AEEF0A3EFF0900132E090014DF090F0
:106BE900015AE0B40006A3E0B40001D35003026CDB
:106BF900F9E4FCFD90015AE0FEA3E0FF121491C0F4
:106C090004C005C006C007900141121285C004C026
:106C190005C006C0079000D5E0FB7A00E433E450D4
:106C29000114FCFDAE02AF03121454C004C005C028
:106C390006C007E4FCFD900110E0FEA3E0FF12147A
:106C490091C004C005C006C0077C6F7D127E837F9A
:106C59003A12112C12112C121522BFFF02800302C5
:026C69006CF9C4
:106C6B0090015AE0FAA3E0FB900129EAF0A3EBF0C4
:106C7B001251E29000D6E0FAA3E0FB900125EAF076
:106C8B00A3EBF0900135E0FAA3E02401FBE43A908A
:106C9B000127F0A3EBF090011DE0FF129CBAEE90E0
:0D6CAB00012DF0A3EFF0900116E0B4011DE3
:106CB80090010DE0FBE4900133F0A3EBF074059034
:0D6CC800014FF0900135E4F0A3F00291D0EF
:106CD50012965FE4900149F0740A90014FF0E49038
:106CE5000151F004900150F0900133E4F0A37404D5
:106CF500F0025F0FE4FCFD90015AE0FEA3E0FF12F5
:106D05001491C004C005C006C00790014112128548
:106D1500C004C005C006C0077466FEFCFD743FFFD5
:066D2500121522BFFF6BF6
:106D2B0012965F1251E2E4900149F0740A90014F00
:106D3B00F0E4900151F07404900150F09000D6E013
:106D4B00FAA3E0FB900125EAF0A3EBF0900135E00C
:106D5B00FAA3E02401FBE43A900127F0A3EBF090B7
:106D6B00015AE0FAA3E0FB900129EAF0A3EBF090C3
:106D7B00011DE0FF129CBAEE90012DF0A3EFF090F5
:106D8B000133E4F0A37404F0025F0F9000D6E0FA35
:106D9B00A3E0F4FBEAF4FA0BEB70010AC002C003A8
:106DAB007B027A0079E17D057C5578B512081D15BB
:106DBB0081158190010BE06401600A9000DEE0B464
:056DCB000101D340109E
:106DD0007B027A0079E39000DEE0FD1293FF8017DA
:106DE00074449000E4F014A3F0743AA3F090010B03
:106DF000E024309000E7F090012FE0FA7404C39A89
:106E00009000E1F07406A3F07F017B027A0079E143
:0C6E10001295A9900152E06003026F216E
:106E1C00900135E06003026EA5A3E0707C90013216
:106E2C00E0FBE4C0E0C003FCFD900154E0FEA3E0F5
:106E3C00FF121491C004C005C006C00790013D129A
:106E4C001285C004C005C006C0077C6F7D127E830E
:106E5C007F3A12112CC004C005C006C007E4FCFD2B
:106E6C0090015AE0FEA3E0FF121491C004C005C0CB
:106E7C0006C007900141121285C004C005C006C0AF
:106E8C00077B027A0079E17D057C5578C612081DD6
:106E9C0074F62581F581026F77900135E0C0E0A38F
:106EAC00E0C0E0E4FCFD900154E0FEA3E0FF12140E
:106EBC0091C004C005C006C00790013D121285C0E8
:106ECC0004C005C006C0077C6F7D127E837F3A121A
:106EDC00112CC004C005C006C007E4FCFD90015A8B
:106EEC00E0FEA3E0FF121491C004C005C006C00769
:106EFC00900141121285C004C005C006C0077B0278
:106F0C007A0079E17D057C5578D912081D74F62537
:056F1C0081F5818056A3
:106F2100E5FDFF7E00E4FC7D6412013DE4FC7DFF94
:106F3100120151C006C007E4FCFD9001A8E0FEA3C8
:106F4100E0FF121491C004C005C006C007900141C2
:106F5100121285C004C005C006C0077B027A007901
:106F6100E17D057C5578EC12081D74FA2581F581C7
:106F710074259000F0F07F027B027A0079E112958E
:106F8100A9025F0FD2B2D2B41251E27F05129CBAAC
:106F9100E4FCFD121491C004C005C006C0079001B5
:106FA10041121285C004C005C006C0077466FEFC0C
:0A6FB100FD743FFF121522BFFF4AD6
:106FBB0012965F1251E2C201E4900149F0740A90FB
:106FCB00014FF0E4900151F07404900150F09001E6
:106FDB005AE0FAA3E0FB900129EAF0A3EBF0900151
:106FEB001DE0FF129CBAEE90012DF0A3EFF0900183
:106FFB0033E4F0A37404F0025F0F90014CE0B40192
:0F700B0007900133E4F0A3F090014CE0B402567B
:10701A007B057A5579FE129308EF640160030291A9
:01702A00D095
:10702B007F05129CBAEE900129F0A3EFF090011DA1
:10703B00E0FF129CBAEE90012DF0A3EFF01251E29B
:10704B0012965FE4900149F0740A90014FF0E490BE
:10705B000151F07402900150F0900133E4F0A374ED
:10706B0004F0025F0F7B027A0079E17D057C567894
:10707B000F12081D7B027A0079E99000DEE0FD1209
:10708B0093FF74069000E1F07F017B027A0079E1B7
:10709B001295A9900133E0C0E0A3E0C0E07B027A37
:1070AB000079E17D057C55783712081D1581158116
:0D70BB0074029000E1F0900130E0B4010A91
:0A70C80074079000E2F0C2B38002EA
:1070D200D2B37F027B027A0079E11295A990013343
:0D70E200E06003027A91A3E06003027A915E
:1070EF00900139120089E4FCFD74A0FE7441FF1277
:1070FF00112C121495EE90015EF0A3EFF090011396
:10710F00E0FEA3E0FFE4FCFD121491C004C005C033
:10711F0006C0077C6F7D127E837F3A12112CC0044C
:10712F00C005C006C0079000D5E0FD7C00E4C0E0BC
:10713F00EDFFD0E0FE33E4500114FDFC12145412A5
:10714F00112CC004C005C006C007900141121129BF
:10715F00121495EE900162F0A3EFF09000DEE07054
:10716F005F900117E0FF7E00E433E4500114FCFD53
:10717F00121454C004C005C006C0077C6F7D127E78
:10718F00837F3A12112CC004C005C006C0079001BE
:10719F0041121129C004C005C006C0079000D5E0F8
:1071AF00FD7C00E4C0E0EDFFD0E0FE33E4500114BD
:1071BF00FDFC12145412112C121495EF900145F08E
:1071CF009000DFE0FEA3E0FFE4FCFD121491C00489
:1071DF00C005C006C0077C6F7D127E837F3A1211F7
:1071EF002CC004C005C006C0079000D5E0FFE4FE28
:1071FF0033E4500114FDFC12145412112CC004C0BE
:10720F0005C006C007900141121129121495EE9086
:10721F000158F0A3EFF09000D5E0FF7E00E433E4D7
:10722F00500114FCFD121454C004C005C006C00761
:10723F007CEC7D517EB87F3F12112CC004C005C07D
:10724F0006C007900141121129121495EE900164A6
:10725F00F0A3EFF0900141120089E4FEFCFD743FB2
:10726F00FF12112C121495EE900168F0A3EFF0901D
:10727F00011DE0B4046DE4FCFD9000DFE0FEA3E02F
:10728F00FF121491C004C005C006C0077C6F7D12A9
:10729F007E837F3A12112CC004C005C006C0079030
:1072AF0000D5E0FF7E00E433E4500114FCFD12141E
:1072BF005412112CC004C005C006C007E4FCFD74B5
:1072CF00C0FE743FFF120FD5C004C005C006C00733
:1072DF00900141121129121495EE90015CF0A3EF69
:1072EF00F0801D900141120089E4FCFD7428FE74AA
:1072FF0041FF12112C121495EE90015CF0A3EFF0E8
:10730F009000DAE0FAA3E0BA0004B40001D3405DC4
:10731F009000D3E0FEA3E0FFE4FCFD121491C00443
:10732F00C005C006C007E4FCFD7480FE743FFF1269
:10733F00112CC004C005C006C0079000DAE0FEA300
:10734F00E0FFE4FCFD121491121288C004C005C0C6
:10735F0006C007E4FCFD7461FE7445FF12112C1288
:0D736F001495EE900137F0A3EFF00274D4F6
:10737C00900113E0FAA3E0BA0704B46C01D3507483
:10738C009000D3E0FAA3E0FBE4FCFDAE02AF0312E5
:10739C001491C004C005C006C007E4FCFD7480FE57
:1073AC00743FFF12112CC004C005C006C00790002A
:1073BC00D3E0FEA3E0FFE4FCFD121491C004C00571
:1073CC00C006C0077CCD7DCC7E4C7F3E12112C12AA
:1073DC001288C004C005C006C007E4FCFD7461FE41
:1073EC007445FF12112C121495EE900137F0A3EF97
:0473FC00F00274D453
:107400009000D3E0FAA3E0FBBA0103B42C00406C77
:10741000E4FCFDAE02AF03121491C004C005C00627
:10742000C007E4FCFD7480FE743FFF12112CC00401
:10743000C005C006C0079000D3E0FEA3E0FFE4FC57
:10744000FD121491C004C005C006C00774CDFC1421
:10745000FDFE743DFF12112C121288C004C005C03D
:1074600006C007E4FCFD7461FE7445FF12112C1286
:107470001495EE900137F0A3EFF080589000D3E020
:10748000FAA3E0FBE4FCFDAE02AF03121491C004CA
:10749000C005C006C007E4FCFD7480FE743FFF1207
:1074A000112CC004C005C006C0077CCD7DCC7E4C2D
:1074B0007F3D12112CC004C005C006C007E4FCFDCE
:1074C0007461FE7445FF12112C121495EE90013771
:1074D000F0A3EFF0900137E0FAA3E0FB9001AEEAF1
:1074E000F0A3EBF09000DEE0FA64026009EA6403C6
:1074F0006004EAB4042D9001391200899000D5E0AF
:10750000FF7E00E4FC7D5012013DEE33E450011497
:10751000FDFC12145412112C121495EE900160F01F
:10752000A3EFF09000DEE0B4053A9000D3E0FEA3B4
:10753000E0FFE4FCFD121491C004C005C006C007C2
:107540007C297D5C7E8F7F3D12112CC004C005C05C
:1075500006C007900139121129121495EE900160AE
:10756000F0A3EFF09000DEE0B40101D3404BE4FC67
:10757000FD900160E0FEA3E0FF121491C004C0057D
:10758000C006C007900139120089E4FCFD74A0FE1A
:107590007442FF12112C121522BFFF1D90013912E7
:1075A0000089E4FCFD74A0FE7442FF12112C121439
:1075B00095EE900160F0A3EFF09000DEE0B40101E1
:1075C000D34006740190010BF0E4900147F0A3F062
:1075D000C20290014AF0900152F07960F309F37908
:1075E00062F309F3A3F0900118E0B40001D3500353
:0375F000027724FB
:1075F3007F0D1296DB7F0A1296DB7B027A0079E11C
:107603007D057C56782112081D7B027A0079E112F0
:1076130096EA7B027A0079E17D057C55785D120854
:107623001D7B027A0079E19000DEE0FD1293FF7B7F
:10763300027A0079E11296EA9000D3E0C0E0A3E079
:10764300C0E07B027A0079E17D057C5578651208FC
:107653001D158115817B027A0079E11296EA90006B
:10766300D5E0FBE4C0E0C0037B027A0079E17D054D
:107673007C55787812081D158115817B027A007973
:10768300E11296EA9000DAE0FEA3E0FFE4FCFD12CB
:107693001491C004C005C006C0077C6F7D127E83B1
:1076A3007F3A12112CC004C005C006C0077B027AC2
:1076B3000079E17D057C56783312081D74FC258121
:1076C300F5817B027A0079E11296EA900160E0C0CD
:1076D300E0A3E0C0E07B027A0079E17D057C567887
:1076E3004512081D158115817B027A0079E11296F6
:1076F300EA900137E0C0E0A3E0C0E07B027A0079C2
:10770300E17D057C56785612081D158115817B0293
:107713007A0079E11296EA7F0D1296DB7F0A1296C0
:10772300DB9000DAE0FAA3E0FBBA0004B40001D373
:027733004064B0
:10773500900139120089E4FCFDAE02AF03121491E9
:1077450012112C121495EE900156F0A3EFF0900053
:10775500D6E4F0A3F0C0E0C0E07461C0E07445C0B9
:10776500E09000DAE0FEA3E0FFE4FCFD12149112C4
:107775001288C004C005C006C007E4FCFD74C8FE3D
:107785007442FF12112C121495EE9000D8F0A3EF5D
:04779500F002791273
:10779900900113E0FAA3E0BA0704B46C01D34003E3
:0377A90002784320
:1077AC009000D3E0FAA3E0FBE4FCFDAE02AF0312C1
:1077BC001491C004C005C006C0077CCD7DCC7E4CA6
:1077CC007F3E12112CC004C005C006C007900139C1
:1077DC00121129121495EE900156F0A3EFF09000BF
:1077EC00D6E4F0A3F0C0E0C0E07461C0E07445C022
:1077FC00E09000D3E0FEA3E0FFE4FCFD121491C086
:10780C0004C005C006C0077CCD7DCC7E4C7F3E12EB
:10781C00112C121288C004C005C006C007E4FCFD80
:10782C0074C8FE7442FF12112C121495EE9000D8FD
:07783C00F0A3EFF002791246
:107843009000D3E0FAA3E0FBBA0103B42C00500389
:037853000278E6D2
:10785600E4FCFDAE02AF03121491C004C005C006DD
:10786600C00774CDFC14FDFE743DFF12112CC0043C
:10787600C005C006C007900139121129121495EEF1
:10788600900156F0A3EFF09000D6E4F0A3F0C0E02C
:10789600C0E07461C0E07445C0E09000D3E0FEA390
:1078A600E0FFE4FCFD121491C004C005C006C00749
:1078B60074CDFC14FDFE743DFF12112C121288C00B
:1078C60004C005C006C007E4FCFD74C8FE7442FF90
:1078D60012112C121495EE9000D8F0A3EFF0802C24
:1078E600900139120089E4FCFD74A0FE7441FF1278
:1078F600112C121495EE900156F0A3EFF09000D6DD
:10790600E4F0A3F0A37446F0A37450F0C2B375FE7E
:107916000175EE0175DE42D2DEC203900139120016
:1079260089E4FCFD7448FE7442FF12112C12149572
:10793600EE9001AAF0A3EFF09000D3E0FEA3E0FFE3
:10794600E4FCFD121491C004C005C006C0077CCD3E
:107956007DCC7E4C7F3D12112CC004C005C006C0F4
:1079660007900139121129121495EE9001ACF0A37B
:10797600EFF0E4FCFD9001ACE0FEA3E0FF121491F1
:10798600C004C005C006C007900139121285C004A4
:10799600C005C006C007E4FCFD74A0FE7441FF12DA
:1079A6001522BFFF1D900139120089E4FCFD74A069
:1079B600FE7441FF12112C121495EE9001ACF0A347
:1079C600EFF07B027A0079E17D057C567863120838
:1079D6001D74069000E1F07F017B027A0079E112C6
:1079E60095A97F027B057A5579A41295A97F011284
:1079F600956A900156E0FEA3E0FF7D06124911EE5E
:107A0600900154F0A3EFF07F027B057A5579A4121A
:0C7A160095A9E4FF12956AE490014BF082
:107A2200900154E0FCA3E0FD90014BE0FA2AFB2414
:107A32006AF582E43401F583ECF0A3EDF090015A8B
:107A4200E0FCA3E0FDEB247EF582E43401F583EC57
:107A5200F0A3EDF090011DE0FF129CBA90014BE003
:107A6200FA2A2492F582E43401F583EEF0A3EFF0D2
:107A720090014BE004F0B40AA7740790014FF09014
:107A820001AEE0FAA3E0FB900137EAF0A3EBF0903D
:107A92000135E4F0A3F0900132F0025F0FC2B3901F
:107AA200014CE064016004E0B403067405900152E5
:0B7AB200F09000D8E0705DA3E0705978
:107ABD009000D7E004F09000D67003E004F0E4C02D
:107ACD00E0C0E07461C0E07445C0E0E4FCFD9001ED
:107ADD0054E0FEA3E0FF121491C004C005C006C01F
:107AED0007900139121285121288C004C005C00614
:107AFD00C007E4FCFD74C8FE7442FF12112C121471
:107B0D0095EE9000D8F0A3EFF0900137E07004A34C
:107B1D00E060199000D3E0FAF5F0A3E0FB9000D6F9
:0C7B2D00E0B5F006A3E0B50301D3406D05
:107B39001251E212965F7403900149F0740A9001A0
:107B49004FF0E4900151F0900150F09000D6E0FA26
:107B5900A3E0FB900121EAF0A3EBF0900135E0FAF4
:107B6900A3E0FB900123EAF0A3EBF090015AE0FABD
:107B7900A3E0FB900129EAF0A3EBF07962A3E3F01B
:107B890009A3E3F090011DE0FF129CBAEE90012DCC
:107B9900F0A3EFF0900133E4F0A37404F090014CEA
:097BA900E0B402028003027C3A00
:0E7BB2007B057A5579FE129308EF6401707A14
:107BC0001251E212965F740190010BF0E4900149AA
:107BD000F0740A90014FF0E4900151F074029001AA
:107BE00050F09000D6E0FAA3E0FB900121EAF0A368
:107BF000EBF0900135E0FAA3E02401FBE43A9001B8
:107C000023F0A3EBF090015AE0FAA3E0FB900129E6
:107C1000EAF0A3EBF07962A3E3F009A3E3F09001AB
:107C20001DE0FF129CBAEE90012DF0A3EFF0900141
:107C300033E4F0A37404F0025F0F300303027DF518
:107C4000900132E0F5F090014DE065F07003027FA5
:017C5000D063
:107C5100900152E0B40001D34003E014F07F071219
:107C6100504BEE90017AF0A3EFF09001B0120100B9
:097C710000000000E490014BF05A
:107C7A0090014BE025E0246CF582E43401F583E0C1
:107C8A00FCA3E0FD90014BE0FA2AFF246AF582E4A6
:107C9A003401F583ECF0A3EDF09001B0120089EF06
:107CAA00246AF582E43401F583E0FEA3E0FFE4FCF4
:107CBA00FD1201289001B01200D090014BE004F0AF
:107CCA00B408AD75F0039001B01200C412000E9012
:107CDA000154EEF0A3EFF0A3E0FEA3E0FFE4FCFD05
:107CEA00121491C004C005C006C0077C0A7DD77E65
:107CFA00A37F3C12112C121495EE900166F0A3EFAB
:107D0A00F0900154E0FCA3E0FDA3E0FAA3E0FB90AD
:107D1A000167E0F8EBC398FB900166E0F8EA98FA8D
:107D2A00F5F0ECB5F004EDB50300401EE0FAA3E06F
:107D3A00FB900157E02BFB900156E03AFAF5F0EC84
:0A7D4A00B5F005EDB50301D34015B7
:107D5400900156E0FEA3E0FF7D07124911EE900169
:107D640054F0A3EFF0125093EE90018EF0A3EFF0D5
:0F7D74009001B012010000000000E490014BF0FC
:107D830090014BE025E02480F582E43401F583E0A3
:107D9300FCA3E0FD90014BE0FA2AFF247EF582E488
:107DA3003401F583ECF0A3EDF09001B0120089EFFC
:107DB300247EF582E43401F583E0FEA3E0FFE4FCD6
:107DC300FD1201289001B01200D090014BE004F0A5
:107DD300B408AD75F0039001B01200C412000E9008
:107DE300015AEEF0A3EFF0900132E090014DF00262
:027DF3007FD03F
:107DF500900132E0F5F090014DE065F07003027FEF
:017E0500D0AC
:107E0600900152E0B40001D34003E014F012509305
:107E1600EE90018EF0A3EFF09001B0120100000089
:077E26000000E490014BF0A5
:107E2D0090014BE025E02480F582E43401F583E0F8
:107E3D00FEA3E0FF90014BE0FA2AFD7C00247EF5C5
:107E4D0082E43401F583EEF0A3EFF09001B012005F
:107E5D0089ED247EF582E43401F583E0FEA3E0FF95
:107E6D00E4FD1201289001B01200D090014BE00406
:107E7D00F0B408AC75F0039001B01200C412000EFE
:107E8D0090015AEEF0A3EFF09000DEE0B4052EE481
:107E9D00FCFD900158E0FEA3E0FF121491C004C058
:107EAD0005C006C0077C0A7DD77EA37F3C12112C2E
:107EBD00121495EE900166F0A3EFF0801C90014135
:107ECD001200897C0A7DD77EA37F3B12112C1214E0
:107EDD0095EE900166F0A3EFF090015AE0FCA3E05F
:107EED00FD900158E0FAA3E0FB900167E0F8EBC3C9
:107EFD0098FB900166E0F8EA98FAF5F0ECB5F0041D
:107F0D00EDB50300401EE0FAA3E0FB900159E02B14
:107F1D00FB900158E03AFAF5F0ECB5F005EDB5033C
:047F2D0001D3401329
:107F3100900158E0FEA3E0FF124E98EE90015AF036
:107F4100A3EFF07F0712504BEE90017AF0A3EFF010
:0F7F51009001B012010000000000E490014BF01D
:107F600090014BE025E0246CF582E43401F583E0D8
:107F7000FEA3E0FF90014BE0FA2AFD7C00246AF5A5
:107F800082E43401F583EEF0A3EFF09001B012002B
:107F900089ED246AF582E43401F583E0FEA3E0FF75
:107FA000E4FD1201289001B01200D090014BE004D2
:107FB000F0B408AC75F0039001B01200C412000ECA
:107FC000900154EEF0A3EFF0900132E090014DF0FB
:107FD0009000DEE06009E0B401028003028093902B
:107FE000015EE0FAF5F0A3E0FB900154E0B5F00685
:0B7FF000A3E0B50301D340030280931F
:0F7FFB00900147E004F0B40201D35003028098D4
:10800A007F05129CBAEE900129F0A3EFF01251E21B
:10801A0075FD7F75ED7F75DD42D2DE12965F7401C4
:10802A0090010BF0C201E4900149F0740A90014FEB
:10803A00F0E4900151F07404900150F09000D6E001
:10804A00FAA3E0FB900121EAF0A3EBF0900135E0FE
:10805A00FAA3E02401FBE43A900123F0A3EBF079C0
:10806A006290012BE3F009A3E3F090011DE0FF12F7
:10807A009CBAEE90012DF0A3EFF0900133E4F0A347
:09808A007404F01251E2025F0FD0
:10809300E4900147F09000DEE0FAB40101D350030D
:1080A30002818490015EE0FCA3E0FD900154E0B501
:1080B3000406A3E0B50501D3400302818490015A6D
:1080C300E0FEA3E0FF900168E0FCA3E0FD9001590E
:1080D300E02DFD900158E03CFCF5F0EEB5F005EF26
:0980E300B50501D35003028184AC
:0F80EC00900148E004F0B40201D35003028189EF
:1080FB007F05129CBAEE900129F0A3EFF01251E22A
:10810B0075FD7F75ED7F75DD42D2DE12965F7401D2
:10811B0090010BF0C201E4900149F0740A90014FF9
:10812B00F0E4900151F07404900150F09000D6E00F
:10813B00FAA3E0FB900121EAF0A3EBF0900135E00C
:10814B00FAA3E02401FBE43A900123F0A3EBF079CE
:10815B006290012BE3F009A3E3F090011DE0FF1205
:10816B009CBAEE90012DF0A3EFF0900133E4F0A355
:09817B007404F01251E2025F0FDE
:10818400E4900148F09000DEE06009E0B401028070
:1081940003028247900113E0B40706A3E0B46C0124
:0681A400D34003028247F4
:1081AA00900162E0FAA3E0FB90015AE0B50206A34F
:0A81BA00E0B50301D3500302824236
:0C81C40090014AE004F0B40401D34077BD
:1081D0007F05129CBAEE900129F0A3EFF01251E254
:1081E00012965FE4900149F0740A90014FF0E49018
:1081F0000151F07403900150F09000D6E0FAA3E032
:10820000FB900121EAF0A3EBF0900135E0FAA3E046
:108210002401FBE43A900123F0A3EBF07962900192
:108220002BE3F009A3E3F090011DE0FF129CBAEEEE
:1082300090012DF0A3EFF0900133E4F0A37404F06B
:028240008005B7
:0F824200E490014AF09000DAE0702AA3E0702681
:1082510090015AE0F5F07962E3B5F009A3E0F5F099
:1082610009E3B5F000500F90015AE0FAA3E0FB7961
:1082710062EAF309EBF39000DEE060030283EF9022
:1082810000DAE0B40006A3E0B40001D35003028396
:01829100EFFD
:1082920090015AE0FEA3E0FF900164E0FCA3E0FD40
:1082A200900145E0FB129759EF640160030283EFEE
:0A82B20090010BE0B40101D3407C01
:1082BC00E014F0740290014FF01251E2900125E4A9
:1082CC00F0A3F0A3F0A3F09000D6E0FAA3E0FB90AB
:1082DC000121EAF0A3EBF0900135E0FAA3E02401D0
:1082EC00FBE43A900123F0A3EBF090015AE0FAA3DF
:1082FC00E0FB900129EAF0A3EBF07962A3E3F0092B
:10830C00A3E3F090011DE0FF129CBAEE90012DF05A
:10831C00A3EFF090010DE0FBE4900133F0A3EBF040
:10832C00A3E4F0A3F0900132F0025F0F1251E2903F
:06833C00011BE0B401404A
:1083420012965F75FE0175EE0175DE42D2DE900176
:1083520033740EF0A37410F0740990014FF07F0192
:1083620012956A9001ACE0FEA3E0FF7D081249116C
:10837200EE900154F0A3EFF0E4FF12956A025F0F52
:1083820012965F7401900149F0740A90014FF0E473
:10839200900151F0900150F09000D6E0FAA3E0FB7A
:1083A200900121EAF0A3EBF0900135E0FAA3E0247A
:1083B20001FBE43A900123F0A3EBF090015AE0FABA
:1083C200A3E0FB900129EAF0A3EBF07962A3E3F0CA
:1083D20009A3E3F090011DE0FF129CBAEE90012D7B
:1083E200F0A3EFF0900133E4F0A37404F09000DE08
:1083F200E0FAB4010280030285B59000DAE0B4002D
:0C84020006A3E0B40001D350030285B5CE
:10840E0090015AE0FAA3E0FB7962E3B5020509E3B5
:10841E00B5030050077962EAF309EBF390015AE0D5
:10842E00FEA3E0FF1297CCEF900150F0BF0001D3F6
:05843E0040282002258A
:10844300900133E4F0A37478F0D202900150E0B4C9
:1084530001067402900149F0900150E0B4020674E1
:1084630004900149F0900133E060030285B5A3E075
:0B84730060030285B52002030285B5FE
:0A847E0090010BE0B40101D3407C33
:10848800E014F0740290014FF01251E2900125E4DB
:10849800F0A3F0A3F0A3F09000D6E0FAA3E0FB90DD
:1084A8000121EAF0A3EBF0900135E0FAA3E0240102
:1084B800FBE43A900123F0A3EBF090015AE0FAA311
:1084C800E0FB900129EAF0A3EBF07962A3E3F0095D
:1084D800A3E3F090011DE0FF129CBAEE90012DF08D
:1084E800A3EFF090010DE0FBE4900133F0A3EBF073
:1084F800A3E4F0A3F0900132F0025F0F1251E29072
:06850800011BE0B401407C
:10850E0012965F75FE0175EE0175DE42D2DE9001A8
:10851E0033740EF0A37410F0740990014FF07F01C4
:10852E0012956A9001ACE0FEA3E0FF7D081249119E
:10853E00EE900154F0A3EFF0E4FF12956A025F0F84
:10854E0012965F740A90014FF0E4900151F0900181
:10855E0050F09000D6E0FAA3E0FB900121EAF0A3E0
:10856E00EBF0900135E0FAA3E02401FBE43A900130
:10857E0023F0A3EBF090015AE0FAA3E0FB9001295F
:10858E00EAF0A3EBF07962A3E3F009A3E3F0900124
:10859E001DE0FF129CBAEE90012DF0A3EFF09001BA
:1085AE0033E4F0A37404F09000DEE0B40101D35084
:0485BE00030286D559
:1085C20090015AE0FAF5F0A3E0FB7962E3B5F00519
:1085D20009E3B5030050077962EAF309EBF390016E
:1085E20058E0FAA3E0FBA3E0FCA3E0FDECB5020433
:0985F200EDB5030040072003046D
:1085FB00D202D2032003030286D5900160E0FAA3D6
:10860B00E0FB900154E0B50205A3E0B50300400385
:10861B000286D590015EE0FAA3E0FB900154E0B531
:10862B000206A3E0B50301D350030286D590015A8D
:10863B00E0FCA3E0FD900168E0FAA3E0FB90015998
:10864B00E02BFB900158E03AFAF5F0ECB5F004EDB5
:05865B00B5030050759D
:10866000740190010BF01251E212965FE4900149FF
:10867000F0740A90014FF0E4900151F0900150F035
:108680009000D6E0FAA3E0FB900121EAF0A3EBF022
:10869000900135E0FAA3E02401FBE43A900123F0D5
:1086A000A3EBF090015AE0FAA3E0FB900129EAF075
:1086B000A3EBF07962A3E3F009A3E3F090011DE0DE
:1086C000FF129CBAEE90012DF0A3EFF0900133E47D
:1086D000F0A37404F09001B01201000000000090BB
:1086E000011DE0FF129CBAEE9001A2F0A3EFF0E4AE
:0486F00090014BF0BA
:1086F40090014BE025E02494F582E43401F583E015
:10870400FEA3E0FF90014BE0FA2AFD7C002492F5E1
:1087140082E43401F583EEF0A3EFF09001B012008F
:1087240089ED2492F582E43401F583E0FEA3E0FFB1
:10873400E4FD1201289001B01200D090014BE00436
:10874400F0B408AC75F0039001B01200C412000E2E
:108754009001A8EEF0A3EFF090015CE0F5F0A3E047
:10876400FB9001A8E0B5F005A3E0B50300400302C7
:0287740087FE7E
:0F877600900153E004F0B40401D35003028803D0
:108785001251E212965F740190010BF0E4900149D9
:10879500F0740A90014FF0E4900151F074059001D6
:1087A50050F0900133E4F0A37404F09000D6E0FAA1
:1087B500A3E0FB900121EAF0A3EBF0900135E0FA8C
:1087C500A3E02401FBE43A900123F0A3EBF0900130
:1087D5005AE0FAA3E0FB900129EAF0A3EBF07962F5
:1087E500A3E3F009A3E3F09001A8E0FAA3E0FB906E
:0987F500012DEAF0A3EBF0800570
:1087FE00E4900153F09000D6E0C0E0A3E0C0E07B2F
:10880E00027A0079E17D057C5578B512081D158137
:10881E00158190010BE06401600A9000DEE0B40166
:04882E0001D3401022
:108832007B027A0079E39000DEE0FD1293FF80175D
:1088420074439000E4F004A3F0743AA3F090010B97
:0A885200E024309000E7F020020A55
:0A885C0090012FE09000E1F0800D84
:10886600900130E0B4010674049000E1F0740590C4
:1088760000E2F07F017B027A0079E11295A990016E
:0788860052E06003028AE3E7
:10888D00900135E060030289C0A3E060030289C056
:10889D00E4FCFD900154E0FEA3E0FF121491C0042E
:1088AD00C005C006C007900139121285C004C0056D
:1088BD00C006C007E4FCFD74C8FE7442FF12152209
:1088CD00BF017C900132E0FBE4C0E0C003FCFD90F1
:1088DD000154E0FEA3E0FF121491C004C005C006D0
:1088ED00C007900139121285C004C005C006C0072B
:1088FD007C6F7D127E837F3A12112CC004C005C09F
:10890D0006C00790015AE0FEA3E0FFE4FCFD12143F
:10891D0091C004C005C006C007900141121285C068
:10892D0004C005C006C0077B027A0079E17D057C95
:0F893D005578C612081D74F62581F581028AE16E
:10894C00E4FCFD900154E0FEA3E0FF121491C0047E
:10895C00C005C006C007900139121285121495EF9C
:10896C00900146F0900132E0FBE4C0E0C0039001BE
:10897C0046E0FBE4C0E0C00390015AE0FEA3E0FF38
:10898C00E4FCFD121491C004C005C006C0079001A0
:10899C0041121285C004C005C006C0077B027A00D4
:1089AC0079E17D057C56787412081D74F82581F5E3
:0489BC0081028B3970
:1089C000E4FCFD900154E0FEA3E0FF121491C0040A
:1089D000C005C006C007900139121285C004C00549
:1089E000C006C007E4FCFD74C8FE7442FF121522E5
:1089F000BF017D900135E0C0E0A3E0C0E0E4FCFDF4
:108A0000900154E0FEA3E0FF121491C004C005C021
:108A100006C007900139121285C004C005C006C007
:108A2000077C6F7D127E837F3A12112CC004C00533
:108A3000C006C00790015AE0FEA3E0FFE4FCFD126F
:108A40001491C004C005C006C007900141121285F0
:108A5000C004C005C006C0077B027A0079E17D052D
:108A60007C5578D912081D74F62581F581028B3961
:108A7000E4FCFD900154E0FEA3E0FF121491C00459
:108A8000C005C006C007900139121285121495EF77
:108A9000900146F0900135E0C0E0A3E0C0E0900115
:108AA00046E0FBE4C0E0C00390015AE0FEA3E0FF13
:108AB000E4FCFD121491C004C005C006C00790017B
:108AC00041121285C004C005C006C0077B027A00AF
:108AD00079E17D057C56788612081D74F82581F5AC
:038AE0008180563C
:108AE300E5FEFF7E00E4FC7D6412013DE4FC7DFFB6
:108AF300120151C006C007E4FCFD9001A8E0FEA3EB
:108B0300E0FF121491C004C005C006C007900141E4
:108B1300121285C004C005C006C0077B027A007923
:108B2300E17D057C5578EC12081D74FA2581F581E9
:108B330074259000F0F07F027B027A0079E11295B0
:0E8B4300A9025F0F9000D8E0705DA3E07059AA
:108B51009000D7E004F09000D67003E004F0E4C088
:108B6100E0C0E07461C0E07445C0E0E4FCFD900148
:108B710054E0FEA3E0FF121491C004C005C006C07A
:108B810007900139121285121288C004C005C0066F
:108B9100C007E4FCFD74C8FE7442FF12112C1214CC
:108BA10095EE9000D8F0A3EFF090014CE0B40202F2
:058BB1008003028C3B73
:0E8BB6007B057A5579FE129308EF6401707703
:108BC4001251E212965F740190010BF0E490014996
:108BD400F0740A90014FF0E4900151F07402900196
:108BE40050F09000D6E0FAA3E0FB900121EAF0A354
:108BF400EBF0900135E0FAA3E0FB900123EAF0A347
:108C0400EBF090015AE0FAA3E0FB900129EAF0A30B
:108C1400EBF07962A3E3F009A3E3F090011DE0FF18
:108C2400129CBAEE90012DF0A3EFF0900133E4F022
:108C3400A37404F0025F0F900133E0FAA3E0BA00DA
:0A8C440004B40001D35003028EAA0D
:108C4E00900132E0F5F090014DE065F07003028F77
:018C5E000E07
:108C5F00B2B39001ACE0FEA3E0FF7D07124911EE25
:108C6F00900154F0A3EFF0125093EE90015AF0A33D
:108C7F00EFF09000D6E0C0E0A3E0C0E07B027A0006
:108C8F0079E17D057C56789812081D158115817440
:108C9F00069000E1F07F017B027A0079E11295A93D
:108CAF00E4FCFD900154E0FEA3E0FF121491C00418
:108CBF00C005C006C007900139121285C004C00557
:108CCF00C006C007E4FCFD74C8FE7442FF121522F3
:108CDF00BF017C900135E0C0E0A3E0C0E0E4FCFD03
:108CEF00900154E0FEA3E0FF121491C004C005C030
:108CFF0006C007900139121285C004C005C006C016
:108D0F00077C6F7D127E837F3A12112CC004C00541
:108D1F00C006C00790015AE0FEA3E0FFE4FCFD127D
:108D2F001491C004C005C006C007900141121285FE
:108D3F00C004C005C006C0077B027A0079E17D053B
:0F8D4F007C5578D912081D74F62581F581807145
:108D5E00E4FCFD900154E0FEA3E0FF121491C00468
:108D6E00C005C006C007900139121285121495EF86
:108D7E00900146F0900135E0C0E0A3E0C0E0900124
:108D8E0046E0FBE4C0E0C00390015AE0FEA3E0FF22
:108D9E00E4FCFD121491C004C005C006C00790018A
:108DAE0041121285C004C005C006C0077B027A00BE
:108DBE0079E17D057C56788612081D74F82581F5BB
:108DCE00817F027B027A0079E11295A9900132E04F
:108DDE0090014DF09000DEE06009E0B401028003E6
:108DEE00028EA290015EE0FAF5F0A3E0FB90015432
:0F8DFE00E0B5F006A3E0B50301D34003028EA257
:0F8E0D00900147E004F0B40301D35003028EA795
:108E1C007F05129CBAEE900129F0A3EFF01251E2FB
:108E2C0075FD7F75ED7F75DD42D2DE12965F7401A4
:108E3C0090010BF0C201E4900149F0740A90014FCB
:108E4C00F0E4900151F07404900150F09000D6E0E1
:108E5C00FAA3E0FB900121EAF0A3EBF0900135E0DE
:108E6C00FAA3E0FB900123EAF0A3EBF07962900106
:108E7C002BE3F009A3E3F090011DE0FF129CBAEE86
:108E8C0090012DF0A3EFF0900133E4F0A37404F003
:068E9C001251E2025F0F1B
:088EA200E4900147F00291D0B9
:108EAA0012965F740A90014FF0E4900151F090011C
:108EBA0050F09000D6E0FAA3E0FB900121EAF0A37B
:108ECA00EBF0900135E0FAA3E0FB900123EAF0A36E
:108EDA00EBF090015AE0FAA3E0FB900129EAF0A333
:108EEA00EBF07962A3E3F009A3E3F090011DE0FF40
:108EFA00129CBAEE90012DF0A3EFF0900133E4F04A
:108F0A00A37404F0025F0FD2B2D2B3900150E0B45E
:108F1A0003028050500BE060121460221460328009
:0B8F2A007AE024FC605114606180704C
:108F35007B027A0079E17D057C5678A912081DD25D
:108F4500B4805D7B027A0079E17D057C5678BA12A2
:108F5500081DD2B4804A7B027A0079E17D057C56F2
:108F650078CB12081DC2B480377B027A0079E17D87
:108F7500057C5678DC12081DC2B480247B027A0079
:108F850079E17D057C5678ED12081DC2B480117B10
:108F9500027A0079E17D057C5678FE12081DC2B47F
:108FA50074069000E1F07F017B027A0079E1129569
:108FB500A9900133E0FAA3E0FBBA0004B40401D39D
:108FC5004009900133E4F0A37404F0900133E0709C
:058FD5001EA3E0701A6C
:108FDA0012960B900133E4F0A37404F0900151E06F
:108FEA0004F0B40601D34002E4F0900151E0B40366
:108FFA000302908E500CE0602014604814606502F1
:10900A0091B5E024FC70030290AE14700302911D26
:09901A0014700302917C0291B56F
:10902300900126E0F4FB900125E0F4FA0BEB7001CC
:109033000AC002C0037B027A0079E17D057C577880
:109043000F12081D158115810291B5900127E0C00B
:10905300E0A3E0C0E07B027A0079E17D057C5778EC
:109063002012081D158115810291B5900121E0C0E0
:10907300E0A3E0C0E07B027A0079E17D057C5778CC
:109083003112081D158115810291B5900123E0C0AD
:10909300E0A3E0C0E07B027A0079E17D057C5778AC
:1090A3004212081D158115810291B5900149E060B6
:1090B3000F14601E14602D14603C14604B0291B5B4
:1090C3007B027A0079E17D057C57785312081D02F3
:1090D30091B57B027A0079E17D057C5778641208AB
:1090E3001D0291B57B027A0079E17D057C57787585
:1090F30012081D0291B57B027A0079E17D057C5748
:10910300788612081D0291B57B027A0079E17D050C
:109113007C57789712081D0291B5E4FCFD90012954
:10912300E0FEA3E0FF121491C004C005C006C0070F
:10913300900141121285C004C005C006C007E4FCBB
:10914300FD90012BE0FEA3E0FF121491C004C005C3
:10915300C006C007900141121285C004C005C006B5
:10916300C0077B027A0079E17D057C5778A8120855
:109173001D74F82581F5818039E4FCFD90012DE013
:10918300FEA3E0FF121491C004C005C006C00790FF
:109193000141121285C004C005C006C0077B027AD4
:1091A3000079E17D057C5778BA12081D74FC25818E
:1091B300F5817F027B027A0079E11295A990014C37
:0491C300E0B4020909
:0C91C7001207F5740190014FF0025F0FD9
:1091D300900116E0B401004007E0B40301D3400658
:1091E3007401900116F090011DE0B40401D3400313
:1091F3007404F0900113E0FAA3E0FBBA0603B44051
:10920300004009BA0704BB6C01D3400A90011374F0
:1092130007F0A37476F0900109E0FAA3E0FBBA012A
:1092230003B4F4004009BA0904BBC401D3400A9053
:1092330001097404F0A374B0F090011EE0FAA3E0F6
:10924300FBBA0703B4D0004009BA0B04BBB801D37F
:10925300400A90011E7408F0A37484F0900110E09A
:10926300FAA3E0FBBA0103B4F4004009BA0404BB57
:10927300B001D3400A9001107403F0A374E8F09096
:109283000117E0B405004007E0B41901D3400674A8
:109293000F900117F0900120E0B40101D340037453
:1092A30001F090011AE0B41E00400AE0FB7A00B41A
:1092B300F001D34006743C90011AF090010DE0B424
:1092C3001E00400AE0FB7A00B4F001D34006743C70
:1092D30090010DF090010EE0FAA3E0FBBA0103B494
:1092E300F4004009BA0904BBC401D3400A90010E3B
:1092F3007404F0A374B0F0900118E0B40101D340FA
:05930300037401F022DB
:109308007841EBF208EAF208E9F21207F5741990CD
:1093180001B4F0900130E024FF92047F017941E329
:10932800C0E009E3C0E009E3F9D002D0031295A92F
:109338007B027A0079E17D057C5778CC12081D7490
:10934800069000E3F0E49001B5F0A3F09001B6E0D8
:07935800640270030293E1BF
:10935F00900120E0B40103120003129672EF900106
:0A936F00B6F064016004E0B40329C5
:079379009001B5E0B4011002
:10938000E4F074069000E3F074209000EAF080129C
:1093900074019001B5F074209000E3F07406900021
:1093A000EAF07F027B027A0079E11295A990013000
:1093B000E0B4010874079000F0F08006742090007B
:0E93C000F0F0A204E433FA900130E06A608617
:1093CE00E024FF92049001B4E014F0600302935481
:0993DE00E4FF229001B5E0FF223A
:1093E7004E6943444E694D484C6946654C69496F1F
:0893F7004C69506F534C4120FA
:1093FF007844EBF208EAF208E9F28D07E49001B73E
:01940F00F06C
:10941000EF25E025E0FE9001B7E02E9093E793FE64
:109420007944E3FD09E3FC09E3F8EE1200267946EE
:10943000E304F3197003E304F39001B7E004F0B41C
:0394400004CE2235
:10944300900121E4F0A3F0A3F0A3F0A3F0A3F0A311
:10945300F0A3F0A3F0A3F0A3F0A3F0A3F0A3F022F2
:0B946300EEB40005EFB40001D3400799
:08946E00EF1F70F11E80EE22D9
:10947600C283E4FE7F641294637F331294E07F32EA
:109486001294E07F281294E07F0C1294E07F06127B
:0F94960094E07F011294E07E017FF41294632230
:1094A5008F0553800FED54F04280D283E4FE7F3266
:1094B500129463C28353800FEDC454F04280D2836B
:1094C500E4FE7F32129463C2837E017FF4129463BB
:0194D5002274
:0A94D6007847EFF2D2821294A5222B
:0A94E0007848EFF2C2821294A52230
:1094EA000E1F111111111F000E1F1111111F1F0044
:1094FA000E1F11111F1F1F000E1F111F1F1F1F00FC
:10950A000E1F1F1F1F1F1F000002060E060200006B
:10951A0000080C0E0C080000001F1517111F000090
:10952A00001F10101010101F001F00000000001F65
:10953A00001F01010101011F001F1F1F1F1F1F1F05
:10954A000E1F11111F1F1F000002060E0602000047
:10955A0000080C0E0C080000001F1517111F000050
:10956A007849EFF27440794AF37949E375F040A4F7
:07957A007949F3E4794BF39A
:10958100794AE3FF1294E07949E3FA784BE22A90B1
:1095910094EA93FF1294D6794AE304F3794BE304F6
:0895A100F3794BE3B440D92239
:1095A900784CEFF2784DEBF208EAF208E9F2EF14A1
:0C95B900600A14600E1460121460162288
:1095C5007F801294E080137FC01294E0800C7FFFAF
:0E95D5001294E080057FFF1294E0E47950F3D9
:1095E300794DE3FD09E3FC09E3F812005EFF1294F1
:1095F300D6794FE304F3197003E304F37950E304DA
:08960300F37950E3B410D92201
:07960B0090011CE0B40121F5
:04961200E47953F3B1
:10961600C2B5E4FE7F28129647D2B5E4FE7F3C121F
:0E96260096477953E304F37953E3B406E32245
:0796340090011CE0B4010BE2
:0C963B00C2B5E4FE7F3C129647D2B52277
:04964700EE4F60136F
:10964B007B007A06DBFEDAFC7C06E4FDEF1F70EC98
:04965B001E80E92262
:07965F0090011CE0B4010BB7
:0C966600C2B57E037F20129647D2B522C9
:10967200E47955F3208004047955F32081057402BE
:109682007955F320800820810574037955F37955C3
:0C969200E360031296343080032081292D
:10969E00E4FE7F321296477954E3B40F01D34012A1
:0696AE007955E3B4020748
:1096B400E47954F37F04227955E3FF227954E304D7
:0C96C400F380D1E47954F37955E3FF22E0
:0B96D0007951E39001B8F0C205FF22C1
:0F96DB002006FDEF7952F3D206300702D2992212
:1096EA007856EBF208EAF208E9F27956E3FD09E363
:0B96FA00FC09E3F812005E642460210C
:109705001200037956E3FD09E3FC09E3F812005E54
:10971500FF1296DB7958E304F31970D3E304F38061
:02972500CE2252
:0A972700C0E0C0D0E9C00130980D89
:0D973100C298E5997951F3D205C2988014D1
:03973E0030060DE5
:0D974100C2067952E3F599C299C20780046F
:0B974E00C299D207D001D0D0D0E03289
:109759007878EEF208EFF2787AECF208EDF2787C9C
:10976900EBF27962E38EF0B5F00709E38FF0B5F01B
:0397790000500D90
:0D977C00E4797DF37962EEF309EFF38040AC
:109789007879E2FF7963E3C39FFF18E2FB19E39B52
:10979900FE12020EEF797DF3797CE3F5F0787DE234
:1097A900B5F001D3401A787AE2F5F07978E3B5F0AB
:1097B9000A08E2F5F009E3B5F001D340037F01227D
:0397C900E4FF2298
:1097CC00787EEEF208EFF2900135E0FAA3E0FB7937
:1097DC0059E3FD7C00E4B502098BF0ED6B700302DC
:0E97EC00996DBA0004BB0001D3500302996DC1
:1097FA00EB7959F3129970900135E0FAA3E0BA00B7
:06980A0003B40600501E2D
:04981000E47980F384
:109814007980E3FA2A246EF8E4F208F27980E3040A
:0F982400F37980E3B405E9E4FF2274057980F35A
:109833007980E3FB25E0246AF8EB25E0246CF9E268
:10984300F30809E2F37980E314F37980E3B40001C8
:10985300D350DD1299C4EE796EF309EFF39001183A
:07986300E0B40001D3400056
:0E986A00900135E0B40005A3E0B40A005010F0
:10987800795EE4F3097463F3795CE4FFF309F32296
:0C988800795AE4F3097463F3E47980F387
:109894007880E2FA2A246EF8795AE3F5F0E2B5F01A
:0C98A4000909E3F5F008E2B5F000500DF2
:1098B000EA2A246EF8795AE2F30809E2F37980E3A0
:1098C00004F37980E3B405CC900118E0B40001D32F
:0298D000400056
:1098D200795EE3701909E37015785CE2701008E2B2
:0B98E200700C785AE2700708E2700377
:1098ED007F0222795EE3F5F0785AE2B5F00909E3DB
:0998FD00F5F008E2B5F00050128C
:10990600795A785EE3F20908E3F2795CE4FFF30939
:0B991600F322795CE3701109E3700D8F
:10992100796E785CE3F20908E3F2E4FF22795CE303
:10993100F5F0786EE2B5F00909E3F5F008E2B5F06B
:0399410000400DD6
:10994400796E785CE3F20908E3F2E4FF22785FE2DF
:10995400FA795DE3C39AFB18E2FC19E39CB40004B2
:06996400BB0201D3400329
:06996A007F0122E4FF2250
:109970007881EEF208EFF27960E3700C09E3700889
:0A9980007960EEF309EFF3227F0592
:10998A00EF25E02460F8EF25E02462F9E2F3080904
:10999A00E2F3DFEC7861E2FA7982E3C39AFF18E234
:1099AA00FB19E39BFE12020EEE7964F309EFF379D9
:0A99BA00817860E3F20908E3F2226D
:1099C4007967E3FB19E3FAEBC333CA33CAFB79655E
:1099D400E32BFB19E33AFA7968E3FC09E3FDE4FEBF
:1099E4007F0312013DEB2FFFEA3EFE786BE2FB188A
:1099F400E2FAEBC333CA33CAFBEF2BFBEE3AFA7835
:109A04006DE22BFF18E23AFEE4FCFD121491C0044F
:109A1400C005C006C0077C397D8E7EE37F3D1211F0
:109A24002C121495EE7883F208EFF218E2FE08E2A5
:029A3400FF220F
:099A3600C2A3C2A2D2A1D2A02257
:109A3F007885ECF208EDF29001B97403F0A374E8A5
:109A4F00F0D2A3EF2400FBEE34057987F309EBF393
:109A5F0019E3FE09E3FF129BA07985E3FE09E3FFFB
:099A6F00129BFF129C5CC2A322B1
:109A78009001B97401F0A3742CF0D2A3EF2400FB79
:109A8800EE34067989F309EBF319E3FE09E3FF12D3
:109A98009BA0129AADEE798BF309EFF3C2A319E3F9
:059AA800FE09E3FF22AE
:109AAD00798DE4F309F3798FF309740FF3798FE36B
:079ABD006480B48000403D0D
:109AC400129C86A2A0E4335401FBE47991F309EBE0
:109AD400F37890E2FAE3FD19E3FC0AED8005C33361
:109AE400CC33CCDAF9FD798EE34DF319E34CF379F9
:109AF40090E314F3F41970BEE314F380B9798DE3A1
:059B0400FE09E3FF2251
:109B09009001B97403F0A374E8F0D2A37E047FC076
:069B1900129BA0C2A32272
:109B1F009001B97403F0A374E8F0D2A37E047F80A0
:099B2F00129BA0129C5CC2A3224F
:109B38007893EEF208EFF29001B97403F0A374E899
:109B4800F0D2A37E047F40129BA07993E3FE09E341
:0A9B5800FF129BFF129C5CC2A322C7
:109B62009001B97403F0A374E8F0D2A3EF2400FBD0
:109B7200EE34077995F309EBF319E3FE09E3FF12DB
:089B82009BA0129C5CC2A3220F
:109B8A009001B97403F0A374E8F0D2A37E04E4FF51
:069B9A00129BA0C2A322F1
:109BA0007897EEF208EFF27999E4F309740AF37901
:099BB00099E36480B48000404395
:109BB900789AE2FA7998E3FD19E3FC0A8005C31360
:109BC900CD13CDDAF9ED5401FD7C00E4799BF3095D
:109BD900EDF319E3B4000909E3B40104D2A1800249
:109BE900C2A1129C86799AE314F3F41970B8E314AC
:069BF900F380B3C2A122BB
:109BFF00789DEEF208EFF2799FE4F309740FF37991
:099C0F009FE36480B4800040432F
:109C180078A0E2FA799EE3FD19E3FC0A8005C313F4
:109C2800CD13CDDAF9ED5401FD7C00E479A1F309F7
:109C3800EDF319E3B4000909E3B40104D2A18002E9
:109C4800C2A1129C8679A0E314F3F41970B8E31446
:049C5800F380B322C0
:109C5C00C2A39001B9E0FEA3E0FF129CA1D2A374B1
:109C6C00FFFAFB20A013EA6480B48004BB0001D38C
:0A9C7C004007EB1B70ED1A80EA228E
:109C8600D2A29001B9E0FEA3E0FF129CA1C2A2906D
:0B9C960001B9E0FEA3E0FF129CA12238
:109CA100E4FAFB8EF0EAB5F0068FF0EBB5F0005068
:099CB100070BEB70EE0A80EB22B8
:109CBA0078A3EFF29001BC12010000000000E490CA
:039CCA0001BBF0EB
:109CCD00E4FE7FC812946379A3E3FF129D22EE9008
:109CDD0001C0F0A3EFF09001BC120089E4FCFD90EF
:109CED0001C0E0FEA3E0FF1201289001BC1200D0DC
:109CFD009001BBE004F0648070C675F007A31200FC
:109D0D00C412000E9001C0EEF0A3EFF09001C0E080
:059D1D00FEA3E0FF229F
:109D2200EF441823232354F8FFD2A40000D2A70043
:079D320000C2A700007E053E
:109D3900C2A4EF30E704D2A68002C2A6EFC333FF64
:109D49000000D2A40000DEE8D2A6C2A40000D2A47A
:0A9D59000000C2A400007F007E0598
:109D6300EFC333FF30A5034401FFD2A40000C2A414
:0E9D73000000DEECEF540FFC7D007F007E0848
:109D8100EFC333FF30A5034401FFD2A40000C2A4F6
:0D9D91000000DEECEF2DFFE43CFED2A72227
:00000001FF
